:020000040800F2
:10300000008000204DDF0008B9E60008BBE600089C
:1030100000000000000000000000000000000000B0
:10302000000000000000000000000000BDE60008F5
:103030000000000000000000BFE6000809B600081C
:1030400081DF000883DF000885DF000887DF0008D4
:1030500089DF00088BDF00088DDF000825EB000802
:1030600091DF000849B6000895DF000897DF0008E7
:1030700099DF00089BDF00089DDF00089FDF000844
:10308000A1DF0008A3DF0008A5DF0008A7DF000814
:10309000A9DF000869B60008ADDF0008AFDF00084F
:1030A000B1DF0008B3DF0008B5DF000859B600083B
:1030B000B9DF0008BBDF0008BDDF0008BFDF000884
:1030C000EDAF16204A62304029BD56B31544E9BF22
:1030D00077900D9CFE0B88C07E2615FA8380734086
:0830E0000FCE674B80D541C003
:1030E80000000000000024400000000000005940DB
:1030F800000000000088C3400000000084D797410A
:103108000080E03779C34143176E05B5B5B89346DB
:10311800F5F93FE9034F384D321D30F94877825AA7
:083128003CBF737FDD4F1575FC
:1031300001000000000000000A0000000000000084
:103140006400000000000000E80300000000000030
:103150001027000000000000A08601000000000011
:1031600040420F0000000000809698000000000020
:1031700000E1F5050000000000CA9A3B00000000D5
:1031800000E40B540200000000E87648170000003D
:103190000010A5D4E800000000A0724E180900003D
:1031A00000407A10F35A00000080C6A47E8D030010
:1031B0000000C16FF286230000008A5D784563013C
:1031C000000064A7B3B6E00D0000E8890423C78AB5
:1031D00010B50124200207490A6802430A6020460C
:1031E00000F00AF8002801D0012010BD08F0F6F91F
:0831F000002010BD0020024088
:1031F800B0B505460E4801780124002916D07D2077
:10320800C00009F03DFD01460A48006809F038FD94
:1032180000F020FE032D09D8002807D10024E04340
:103228002946224600F0DEFD034805602046B0BD71
:0C323800280000202400002014000020CA
:103244000348007803490A68101808607047C046AC
:08325400280000202C000020DE
:0C325C00014800687047C0462C000020AC
:10326800B0B50446FFF7F6FF0546601C02D00448D7
:1032780000780419FFF7EEFF401BA042FAD3B0BD57
:0432880028000020FA
:10328C00F0B587B0044600200690002C75D0059050
:10329C00A06D002807D125465435204604F0F4FAD9
:1032AC0000202870E06501273D072668B068C00043
:1032BC0027D4B0687E4901402943B1607D4800683D
:1032CC007D4909F0DBFC4000801C06900698002824
:1032DC0017D00698401E06900698002811D0069824
:1032EC00401E0690069800280BD00698401E0690AB
:1032FC000698002805D00698401E069006980028CF
:10330C00E7D1B068284208D1A06D10210143A16516
:10331C00E06D012105910843E065B068042101408E
:10332C00A26D102002405118A26D29D103900F20DC
:10333C00C3430493F33B1A40921CA265B268D207B4
:10334C0078D1029027462037226B531E9A411503E1
:10335C00A268237E9B031343627ED1031943A27E92
:10336C0050030843E36803432B430121C807256935
:10337C00002D009009DA854308E0012007B0F0BD6C
:10338C000243A265384607B0F0BD4D052B43387B90
:10339C0045001D43387801280AD1002A13D0A06DAE
:1033AC00012220210143A1651146E06D1043E06527
:1033BC00636A002B01910CD0072080010340A26AA4
:1033CC001A432A4306E008040543636A002B019163
:1033DC00F2D12A46F068394901401143F160387F37
:1033EC0003218F0765682A463A400128E36C0AD10D
:1033FC00206C616C0143A06C084310431843019985
:10340C000843024600E01A4330692D49014011433C
:10341C0031610098854202990CD0BD420AD00198C6
:10342C008007854206D08804054026490A688243F5
:10343C0050190860706907229043656B28437061CE
:10344C00706970218843A16B09010143716127697F
:10345C0001235805874205D0002F0ED1B06A04997C
:10346C00084309E0B06AE06980001C301C2101406F
:10347C00049F8F40206E3843B06270691040A842A0
:10348C000AD10020E065A06D012101430220814397
:10349C00A165059807B0F0BDA06D03990843022102
:1034AC008843A065E06D1843E065012007B0F0BDCE
:1034BC00E8FFFF6F24000020400D03000102DEFF37
:0834CC0002FCFF1F082701406C
:1034D40070B505460068816882680024D20726D04A
:1034E4000222114023D1816805220A40012A16D103
:1034F4008168104A0A40911C816003210160FFF732
:10350400ABFE064628688068C00710D0FFF7A4FE0B
:10351400811B28680329F6D38168C907F3D0A86DF5
:1035240010210143A965E86D01242043E865204684
:0835340070BDC046E8FFFF7FF7
:10353C00F0B581B005460024009400688168C90785
:10354C001AD181682C4A2F32114208D0A86D102153
:10355C000143A965E86D01242043E8650CE081680E
:10356C00254A114001273943816024480068000234
:10357C0005D4687E012825D1204601B0F0BD204835
:10358C000068204909F07AFB401C00900098002844
:10359C00EFD00098401E009000980028E9D00098C9
:1035AC00401E009000980028E3D00098401E009028
:1035BC0000980028DDD00098401E0090009800284C
:1035CC00E7D1D6E7FFF744FE064628680168C9072D
:1035DC00D2D18168C90704D18168074A11403943A7
:1035EC008160FFF735FE811B28680329EED3016843
:1035FC00C907EBD1AAE7C046E8FFFF7F08270140C7
:08360C0024000020400D030022
:10361400F0B581B00E46044601688B6802205B0752
:103624001BD400925422A25C012A16D02746543798
:1036340001253D70C868C0070AD18868C00704D056
:103644008868194A0240901C8860C8682843C8608A
:103654002046FFF771FF002801D001B0F0BDA06D36
:103664001249014028020818A0650020E06521687D
:103674001C220A603870206D0D4A0E4B0E4DC56237
:10368400036342634A68102313434B60403132465C
:10369400009B00F0ADFC21688A68034B13401A1D9F
:1036A4008A6001B0F0BDC046E8FFFF7FFEF0FFFF77
:0C36B4003DE0000833E0000839EA00089F
:1036C000F0B589B0002508955422825C012A02D108
:1036D000022009B0F0BD0646543601243470026859
:1036E00093685B0714D404694B68022B18D104203B
:1036F0000443914884426ED18E48C0430B68D9433D
:103700000143906A084090620024002B74D566E063
:10371000816D20220A4382653570012009B0F0BD19
:103720000796069304263443824B834FBC4267D1ED
:103730000F683B40906A1843906238025369834394
:10374000896801407D480840184350610024002FDB
:1037500004D4079E3570002009B0F0BD01267848DA
:103760003B46076807208205394611407548029399
:10377000834200D082E0F0053B4603407ED1704F8B
:103780003B689343194301433960714800687149AC
:1037900009F07AFA0C2141430C310891089800286D
:1037A000D7D0079E0898401E08900898002823D07C
:1037B0000898401E0890089800281DD00898401EC0
:1037C00008900898002817D00898401E089008987C
:1037D0000028E7D110E00B680024002B0CD55848D6
:1037E0000168594A934265D0584A934265D0554A78
:1037F000934201D105225EE03570204609B0F0BD4C
:10380000029605951F27069C27400F2500950397D4
:10381000BD40046E0195AC4304940F681F4245D02F
:10382000FB07059D2C465AD1BB0753D47B0753D4C5
:103830003B0753D4FB06344651D4BB0662D47B0607
:1038400062D43B0662D4FB0562D40297BB0561D407
:103850007B0561D43B0561D4FB0461D4BB0461D416
:103860007B0461D43B04009C39D4FB035ED4BB03CE
:103870005ED47B03DB1712241C4030E03248029BED
:10388000834203D130063B46034008D02F48029BB9
:10389000834200D05DE7B005074000D059E7284FCC
:1038A0003B68934319430143396052E77B00DC0EC8
:1038B000059D14E00322920501E00322D205114088
:1038C0000722920503689343591801603570002060
:1038D00009B0F0BD012402E0022400E00324039EAD
:1038E000B440049B1C430466069B9B08C069984235
:1038F00000D822E70198C043936A0340B800000F44
:10390000B04018E70524EAE70624E8E70724E6E7DD
:103910000824E4E70924E2E70A24E0E70B24DEE7D1
:103920000C24DCE70D24DAE70E24D8E71024D6E7D0
:103930001124D4E7FFFF07000400008000FFFF0709
:1039400008270140001000B0004000B8002000B47B
:0839500024000020400D0300DB
:10395800F0B58BB0044600210A915420205C012860
:1039680002D102200BB0F0BD089120465430012549
:10397800079005702046FFF7A9FD0646236898685A
:10398800C007A16D42D105950296184608308122DC
:1039980052009143891CA165D968DA68D44F174051
:1039A800DF609A68D34D2A40521918329A60FD4A4E
:1039B8000A4001921946B4310691FB490268002A6F
:1039C8002DD50A9A521C0A920A9A8A4200D982E193
:1039D8000268002A23D50A9A521C0A920A9A8A4235
:1039E80000D978E10268002A19D50A9A521C0A926D
:1039F8000A9A8A4200D96EE10268002A0FD50A9A0B
:103A0800521C0A920A9A8A42D8D964E110200143CA
:103A18000898079A1070A16530460BB0F0BD069A59
:103A280012680768ED4D2F40183503952F4307603E
:103A38007F2504952A400768002F24D50A9F7F1CFC
:103A48000A970A9F8F4200D945E10768002F1AD5C7
:103A58000A9F7F1C0A970A9F8F4200D93BE107689B
:103A6800002F10D50A9F7F1C0A970A9F8F4200D902
:103A780031E10768002F06D50A9F7F1C0A970A9F25
:103A88008F42D8D927E1069D2F680668D34D2E406E
:103A9800039D2E430660049D2F40BA180668002E29
:103AA80024D50A9E761C0A960A9E8E4200D912E1F7
:103AB8000668002E1AD50A9E761C0A960A9E8E4221
:103AC80000D908E10668002E10D50A9E761C0A96D1
:103AD8000A9E8E4200D9FEE00668002E06D50A9E90
:103AE800761C0A960A9E8E42D8D9F4E0069D2E6866
:103AF8000768BA4D2F40039D2F430760049D2E4051
:103B0800B2180668002E24D50A9E761C0A960A9ECC
:103B18008E4200D9DFE00668002E1AD50A9E761C70
:103B28000A960A9E8E4200D9D5E00668002E10D566
:103B38000A9E761C0A960A9E8E4200D9CBE0066839
:103B4800002E06D50A9E761C0A960A9E8E42D8D961
:103B5800C1E0069D2E680768A04D2F40039D2F43A6
:103B68000760049D2E40B2180668002E24D50A9ED0
:103B7800761C0A960A9E8E4200D9ACE00668002E92
:103B88001AD50A9E761C0A960A9E8E4200D9A2E091
:103B98000668002E10D50A9E761C0A960A9E8E424A
:103BA80000D998E00668002E06D50A9E761C0A966B
:103BB8000A9E8E42D8D98EE0069D2E680768874DEA
:103BC8002F40039D2F430760049D2E40B2180668BE
:103BD800002E21D50A9E761C0A960A9E8E427AD815
:103BE8000668002E18D50A9E761C0A960A9E8E42F2
:103BF80071D80668002E0FD50A9E761C0A960A9E72
:103C08008E4268D80668002E06D50A9E761C0A964B
:103C18000A9E8E42DBD95EE0069D2E6807686F4DCE
:103C28002F40039D2F430760049D2E40B21806685D
:103C3800002E21D50A9E761C0A960A9E8E424AD8E4
:103C48000668002E18D50A9E761C0A960A9E8E4291
:103C580041D80668002E0FD50A9E761C0A960A9E41
:103C68008E4238D80668002E06D50A9E761C0A961B
:103C78000A9E8E42DBD92EE0069D2E680768574DB6
:103C88002F40039D2F430760049D2E40B2180668FD
:103C9800002E31D50A9E761C0A960A9E8E421AD8A4
:103CA8000668002E28D50A9E761C0A960A9E8E4221
:103CB80011D80668002E1FD50A9E761C0A960A9E01
:103CC8008E4208D80668002E16D50A9E761C0A96DB
:103CD8000A9E8E42DBD9089807990870A06D1021BA
:103CE800014302208143A16505980BB0F0BDC04691
:103CF800FC7FFFFFE8FFFF7F069909689E68374D44
:103D08002E4001252E439E60049E31408918C90823
:103D18001A69920F29D10F229204314B1B68134064
:103D28009A0C072A21D3D21E012393400993099A9A
:103D380052080992099A002A17D0099A521E099224
:103D4800099A002A11D0099A521E0992099A002A42
:103D58000BD0099A521E0992099A002A05D0099A8D
:103D6800521E0992099A002AE7D1069B1A68049EF6
:103D7800B2430A431A600168184A114002273943BE
:103D88000160FFF767FA069020688168C907029EFC
:103D98000FD1C168019A1143C160A06D012101438F
:103DA800B94335E603800000FFF102008168C907C6
:103DB800EFD0FFF74FFA0699411A20680329F5D387
:103DC8008168C907F2D0A06D10210143A165E06D9B
:103DD8002843E06528460BB0F0BDC046E8FFFF7FEA
:043DE8000827014067
:103DEC00002805D40322034693430A4A9A1803E099
:103DFC000C220240064BD2188007C00E8901C9B2B2
:103E0C008140FF238340106898430843106070473B
:083E1C0014ED00E000E400E0F9
:103E2400002805D41F210840012181400148016078
:083E34007047C04600E100E008
:103E3C00002809D41F21084001218140034801605A
:103E4C00BFF34F8FBFF36F8F7047C04680E100E028
:103E5C00401E010E01D0012070470749074A5060EF
:103E6C00074803680B40032189075918016000209B
:103E7C009060072111607047FFFFFF0010E000E029
:043E8C0020ED00E045
:103E9000B0B5002813D00446407F002803D1207716
:103EA00020460AF0DAF8022060772079002808D04E
:103EB000A168E26820460AF083F8002808D00120B3
:103EC000B0BD20680F49416181681822914381602B
:103ED00000256079002801D0216900E0E9432068CD
:103EE000016181686022914362690A43826081684E
:103EF00080229143A2690A438260012060770020FA
:083F0000B0BDC046B71DC104AD
:103F0800F0B583B0002840D0044606462436022087
:103F18007070276838683049014039602F48803010
:103F2800A0642F483818142108F0AAFE80002B49F5
:103F38004118206401916164FC203840083814213C
:103F480008F09EFE1F210140012528468840E064B4
:103F5800A268E16823690B4361691943A3690B43AC
:103F6800E1691943236A0B433968194311433960DE
:103F78000295A9038A421B4A0AD1002301990B60C2
:103F8800636010601F461D461CE0012003B0F0BDB1
:103F980063683F211940019D29601060581E002365
:103FA80003281F461D460DD8481E810053180021BE
:103FB800D96703210140029D8D400B4805607C3381
:103FC800BC3217460020E06323656765A56530703D
:103FD8000299717003B0F0BD0F80FFFF0008024026
:0C3FE800F8FFFDBF8408024044090240BD
:103FF400F0B582B004462420205C012802D10220BE
:1040040002B0F0BD174625462435012028706A7891
:10401400012A2ED1022068700020E06325682A68F6
:1040240001260196B2432A60A26CE66C5660226DAA
:104034000092002A02D0626DA66D5660226C1C2686
:104044001640019AB2401C4E366816431A4A16604E
:104054006B60A368102B3A4600D00A46AA60102B66
:1040640000D03946E9602968226B002A07D00E2265
:104074000AE0002129708021E16302B0F0BD04222E
:10408400914329602A680A21114329600199090290
:10409400626C1368DB0302D513680B431360009B47
:1040A400002B02D01A680A431A602968019A114346
:0C40B400296002B0F0BDC04604000240CC
:1040C000F0B585B03649091F0E68026813680425EB
:1040D00002932B405F425F410490046C1C232340F9
:1040E000294699400C46039634406042604138436B
:1040F00031D0019201210227029E304638404442CD
:1041000044419F40039D2F420A4600D02146049817
:104110000446243400292FD00820064077427741F6
:10412000DD40280700D53A46002A23D1019A1068BD
:104130000E218843106001252946994018480268DD
:104140000A4302600498C563002121706570416BC9
:1041500000290ED10EE01068800602D41068A84332
:1041600010600F4A1068084310600498016B002922
:1041700000D0884705B0F0BD019B1968890605D4B9
:104180001A680A218A431A60012161700021217096
:10419000034A116839431160C16A0029E9D1E9E78E
:0441A00004000240D5
:1041A400F0B587B00E4668490C78012C02D1022084
:1041B40007B0F0BD0193029203900020059048607F
:1041C4000120087004900404FFF746F805465F4A8E
:1041D4001068C0030AD57D20C700FFF73DF8401BD7
:1041E400B8422FD2594A10682042F6D11068584973
:1041F4004B1C1360084003D053494860049E9EE062
:1042040000930120049080040690106840030BD5AD
:104214007D20C700FFF720F8401BB84212D24B4A5A
:10422400106806990842F5D1039F012F0DD15068FB
:1042340001210143516002983060BFF36F8F0198F0
:10424400706046E00326404979E0506806990843C7
:104254005060EFF31080019072B6059A11460298EF
:1042640043587350731845186F685F60AF689F6058
:10427400EF68DF602F691F616F695F61AF699F61DC
:10428400EF69DF612F6A1F626F6A5F62AF6A9F62C4
:10429400EF6ADF622F6B1F636F6B5F63AF6B9F63AC
:1042A400ED6BDD630F231343403110323F2BD7D323
:1042B400264A1168214208D01168214205D01168AC
:1042C400214202D011682142F3D1019880F3108871
:1042D400039F1646FEF7C0FF05463068204232466B
:1042E4000AD07D20C600FEF7B7FF401BB04220D2A3
:1042F400164A10682042F6D11068009911601449DA
:10430400084003D010494860049E15E01068002658
:10431400069908420BD07D20C400FEF79DFF401B88
:10432400A04206D2094A106806990842F5D1064906
:1043340002E003260449054A5068B84350600598D2
:104344000870304607B0F0BD100F00201020024066
:04435400FA830000E8
:10435800F0B581B0054601200090FEF77BFF0646C8
:10436800244F3868C00318D500980404681C11D07D
:10437800FEF770FF801BA84239D238682042F7D177
:104388000BE03868204208D03868204205D03868E9
:10439800204202D038682042F3D1386816494A1CB6
:1043A8003A60084003D015494860009802E039682F
:1043B800490301D401B0F0BD01218C04691C12D05D
:1043C8000090FEF747FF801BA84210D238682042B1
:1043D800F7D1EAE739682142ECD039682142E9D0BF
:1043E80039682142E6D039682142F3D1E2E7032057
:1043F80001B0F0BD10200240FA830000100F002029
:104408000648C168002901D40020704704490160AA
:1044180004490160C068C00F7047C04608200240C8
:0844280023016745AB89EFCDCC
:10443000F0B581B001200090FEF710FF0446194D41
:104440002868C0030BD5009807047D20C600FEF73E
:1044500005FF001BB0421AD228683842F7D12868FD
:1044600011494A1C2A60084002D0104948600EE0F9
:10447000286840030BD5009887047D20C600FEF70E
:10448000EDFE001BB04202D228683842F7D10098F6
:10449000C0076968014369606868C043C00F01B024
:1044A000F0BDC04610200240FA830000100F00202B
:1044B00006488168490001D4012070470449016021
:1044C0000449016080684000C00F70470C20024022
:0844D0003B2A19087F6E5D4CC8
:1044D800F0B581B001200090FEF7BCFE0446194DEE
:1044E8002868C0030BD5009807047D20C600FEF796
:1044F800B1FE001BB0421AD228683842F7D12868AA
:1045080011494A1C2A60084002D0104948600EE050
:10451800286840030BD5009887047D20C600FEF765
:1045280099FE001BB04202D228683842F7D10098A1
:1045380080076968014369606968014048424841E9
:1045480001B0F0BD10200240FA830000100F0020D7
:10455800F0B583B005462A4C2078012802D1022004
:1045680003B0F0BD029100276760012020707D2014
:10457800C6003046FFF7ECFE002802D0277003B0D3
:10458800F0BD04206860286804280BD11E48801CF0
:104598001C490A6802430A603046FFF7D9FE2770B3
:1045A80003B0F0BDF843029908600021AF68E868DD
:1045B800C01987420191084619D2FC0011490868C0
:1045C800124A10402043104A104308603046FFF753
:1045D800BFFE002808D1A868E968081808347F1CBD
:1045E8008742EBD3019801E002990F60044C054B18
:1045F8001968022291431960019F277003B0F0BD2A
:10460800100F0020142002400200010005E0FEFF08
:10461800F0B583B0364D2978012902D1022003B0C4
:10462800F0BD00266E600121029129700168CA0759
:10463800304F07D043688468C26812042243012BB4
:1046480010D1FA6006220A40062A10D1014610311C
:104658000EC90B43FF208243C143514038680840CC
:10466800184328E03A6106220A40062AEED08A0753
:104678000DD4490720D54169FF229143D2434A40CE
:104688003B683968DBB2AA2B0DD11C460CE03968AF
:10469800194A0A40FF21C94351403B680B40006951
:1046A8001843104307E0BB241140CC2B00D1CC2485
:1046B80080692043084338607D20C4002046FFF706
:1046C80047FE002802D02E7003B0F0BD0196029874
:1046D80046040C3F3868304338602046FFF738FE00
:1046E8003968B143019E39602E7003B0F0BDC046F1
:0C46F800100F00202020024000604F073F
:1047040010B5072101604168012901D0102100E0A2
:104714000C210D4A8B583F241C408460895889021F
:10472400890EC16009494161136812680A408261B7
:10473400D9B2AA2901D10A4603E0BB22CC2900D16F
:10474400CC22026110BDC0462020024000604F0709
:10475400F0B58AB00A68002A00D1BDE00E465F4970
:10476400884201D0052100E0032100910027089729
:1047740009973C46029601900FE01A432A60641C94
:1047840032681146E140BF1C089B1B1D0893099B1E
:1047940008330993002900D19EE001250495A54022
:1047A4002A400792EBD003231846B840C043394649
:1047B40077683A461A40561E012E0697059112D87C
:1047C40006460390019883683340029EF6688E4043
:1047D4001E438660FB06DB0FA3404668AE431E43C0
:1047E4004660039907E0032A0146019803D1029E1B
:1047F4003D46059F1DE0C3680B40029EB568059FBA
:10480400BD401D43C560022A069D12D103911C219F
:10481400089A11400F228A40E3089B00C3181D6ABE
:10482400954332698A4003992A431A6275680322C0
:104834002A40BA4003680B4013430360A903890F5D
:104844009DD01821099A11400F238B40032225463D
:104854009543234A5219156E9D43603205231B0765
:1048640098420AD0204B984205D0204B9842009B96
:1048740004D1022302E0049B00E000238B402B437D
:104884001360174D2A687168CB0208D5079B1A4339
:104894002A606A688B0208D4079B9A4307E0079B47
:1048A4009A432A606A688B02F6D5079B1A436A60AA
:1048B4000C4D6A688B0306D5079B1A436A602A6805
:1048C400C90307D559E7079B9A436A602A68C90355
:1048D40000D552E79A4351E70AB0F0BD000C0050EE
:1048E40000180240801802400004005000080050E4
:1048F400B0B50446074D2868204203D02C602046FA
:1049040009F010FD6868204203D06C60204605F071
:08491400D3FFB0BD0C180240F6
:10491C000120000202490A6802430A607047C0463F
:04492C0000700040D7
:104930000120000202490A6882430A607047C046AB
:0449400000700040C3
:10494400F0B581B0032569021C4E3246143A13684F
:104954008B4303431360012461020022884204D183
:10496400174801683068400502D4002001B0F0BD4A
:104974000092A70206204843124908F083F9201A3E
:10498400022815D03168394215D0012810D0316879
:10499400394210D000280BD0316839420BD0001DA9
:1049A400032805D031683942EAD1009801B0F0BD3E
:1049B400284601B0F0BD009801B0F0BD147000406D
:0849C4002400002040420F0016
:1049CC00F0B587B00125002800D1EEE104950590E3
:1049DC000078C007FA4F2AD0B868F96803252A4630
:1049EC008A433821014010204840821850425041DF
:1049FC00082914D0002812D105984268012001041E
:104A0C008A4208D005231B049A4200D0DAE08204C3
:104A1C003B6813433B603A680A433A60DBE0386812
:104A2C00800304D505984068002800D173E10598EF
:104A3C000078800723D40598007800070CD5B86857
:104A4C0038210140182971D1386E800704D505989A
:104A5C008069002800D15EE1059A1078400700D4E7
:104A6C002EE1B86838210140202974D1F86D8007F7
:104A7C0000D425E19068002800D021E14BE1B96811
:104A8C003820084010214140FA6803252A400223AF
:104A9C005340CA1851425141002820D000291ED140
:104AAC003868059AD168002900D1A2E00721C90213
:104ABC008843116901433960012001023A680A43B5
:104ACC003A608402FEF7C4FB06463868204200D0E8
:104ADC00A1E0FEF7BDFB801B0228F6D965E1396821
:104AEC004905059B03D5D968002900D113E17F2125
:104AFC0009027A688A4359690902114379600028CE
:104B0C000DD10720C0023968814318690843386009
:104B1C0038688004400FAB49C140AB480160AB48DA
:104B2C000068FEF763FB002885D0F4E0386E059929
:104B3C008969002979D0012108433866FEF788FB82
:104B4C000646386E800787D4FEF782FB801B032550
:104B5C000228F6D929E1012003900107F86B0840DF
:104B6C00029006D1F86B0843F863F86B0840069086
:104B7C000698019196480068C00513D40398040266
:104B8C009349086820430860FEF762FB064690488C
:104B9C000068204206D1FEF75BFB801B0325022830
:104BAC00F5D902E1059880688A4C012805D00528C2
:104BBC005AD1F86D04210143F965F86D0399084346
:104BCC00F8655BE03B688B433B6081043B688B433F
:104BDC003B60002A3AD04404FEF73AFB064638689C
:104BEC00204200D023E7FEF733FB801B6428F6D964
:104BFC00DBE001210A02904338608C02FEF728FBAF
:104C0C0006463868204200D115E7FEF721FB801BD1
:104C1C000228F6D9C9E07F20000279688143059803
:104C2C00406900020843786005E701218843386633
:104C3C00FEF70EFB0646386E800700D40CE7FEF735
:104C4C0007FB801B03250228F5D9AEE04404FEF7D0
:104C5C00FFFA06463868204200D1E8E6FEF7F8FA7B
:104C6C00801B6428F6D9A0E0F96D039A9143F9658D
:104C7C00F96D04229143F96500280CD0FEF7E8FA8F
:104C8C000646F86D800713D4FEF7E2FA801B032565
:104C9C00A042F6D989E0FEF7DBFA0646F86D8007EC
:104CAC0006D5FEF7D5FA801B0325A042F6D97CE089
:104CBC0002980028059A03D1F86B01998843F86390
:104CCC00D469002C78D0B86838210140102925D13E
:104CDC00012C20D0F868032101401346126A91423E
:104CEC0019D1702101405A6A914214D17F210902D5
:104CFC0001409A6A120291420DD11F2149040140D0
:104D0C00DA6A9142049D50D1072149070840196B7A
:104D1C0088424AD150E0049807B0F0BD012529061D
:104D2C003868049188433860FEF792FA0646022CE4
:104D3C000BD103956C063868204211D0FEF788FA27
:104D4C00801B03250228F6D92FE06C063868204218
:104D5C002ED0FEF77DFA801B03250228F6D924E01D
:104D6C00F8681E490140059A106A0843516A0143CC
:104D7C00906A00020843D16A126B01431143F96037
:104D8C00386804990843386003980007F9680143B0
:104D9C00F960FEF75DFA0646386820420CD1FEF742
:104DAC0057FA801B03250228F6D9284607B0F0BD18
:104DBC00F86809490140F960002007B0F0BDC04611
:104DCC00001002400024F4002400002014000020F5
:104DDC000070004088130000FCFFFEEF8C80C11FA8
:104DEC00F0B583B00D46012100281BD00191029033
:104DFC007348006807242040A84216D270490868FE
:104E0C00A043284308606F4EFEF722FA07466C4811
:104E1C0000682040A84208D0FEF71AFAC01BB04226
:104E2C00F5D90321084603B0F0BD029E3068810716
:104E3C00654B0CD5410703D521031A680A431A6048
:104E4C000F2109021A688A43B16811431960C0071F
:104E5C001AD15B4800682040A8422AD958490868F2
:104E6C00A04328430860574FFEF7F2F90646544812
:104E7C0000682040A8421CD0FEF7EAF9801BB8421B
:104E8C00F5D9032003B0F0BD706803285CD881000D
:104E9C0001A251588F46C046B54E0008594F000824
:104EAC00634F00086D4F0008194608390968490519
:104EBC0058E0029A10784007434B05D52003196837
:104ECC008143D0680843186018688006400F22D0D0
:104EDC0018683821084008283C4823D01A680A4032
:104EEC00102A5CD1596803220A40032A00D03848A2
:104EFC0059684906490F491C07F0C0FE32494968F8
:104F0C004904490E484330494968490F491C07F088
:104F1C00B5FE2D4B06E01846083800688004410F9A
:104F2C002B48C840196889093C220A4029498958EC
:104F3C001F220A40D0402849086028480068FEF724
:104F4C0055F9004603B0F0BD596D0AE01946083911
:104F5C000968890306E0194608390968890101E0E6
:104F6C00996D8907019900D45CE71968A143014345
:104F7C001960144FFEF76CF9064613480068382187
:104F8C00014002984068C000814200D161E7FEF701
:104F9C005FF9801BB842F0D9032003B0F0BD18684C
:104FAC000840202802D10120C003BBE71868084044
:104FBC00182801D00020B5E77D200002B2E7C046DA
:104FCC0000200240881300000810024000127A00F2
:104FDC000024F40054DE00082400002014000020FB
:104FEC0010B51E4C20688006400F06D02068382172
:104FFC00084008281A4807D110BD083C20688004D6
:10500C00410F1848C84010BD22680A40102A15D11B
:10501C00616803220A40032A00D0124861684906DD
:10502C00490F491C07F02AFE61684904490E4843A0
:10503C006168490F491C07F021FE10BD206808402B
:10504C00202802D10120C00310BD20680840182878
:10505C0001D0002010BD7D20000210BD08100240C0
:08506C0000127A000024F40098
:105074000648006806490968890A1C220A4005494D
:1050840089581F220A40D0407047C046240000209F
:085094000810024094DE000840
:10509C00F0B587B0064680788007564F01D40020C3
:1050AC0050E00596012319073A46183A1068084053
:1050BC00049006D1106808431060106808400690F0
:1050CC0006980292039101931E024B4C20683043C8
:1050DC002060FEF7BDF80546206830420AD1FEF785
:1050EC00B7F8401B0228F7D90320059E0499002924
:1050FC0023D027E0032000900102B8680840059EE9
:10510C0011D0B16988420ED0B86801990904BA6807
:10511C000A43BA60BA688A43BA600146374A1140FA
:10512C00B960C00755D1B86834490840B16901432A
:10513C00B96000200499002904D1029B1968039AD4
:10514C00914319603568E90707D1A9070DD4A90661
:10515C0013D401216A041AD428E03968032291433C
:10516C0072680A433A60A907F1D539680C22914359
:10517C00B2680A433A60A906EBD5032109033A68E1
:10518C008A43F1681143396001216A040ED53A68EB
:10519C001C4B1A40746922433A605A1C944205D144
:1051AC000A043B46483B1C6814431C602A050ED578
:1051BC008C03032292033B689343326913433B6095
:1051CC00A24204D10A04483F39681143396007B040
:1051DC00F0BDFEF73DF80546094CB8688007A2D42F
:1051EC00FEF736F8401BA042F7D900980499002925
:1051FC00A3D0A7E75410024000700040FFFCFFFF53
:08520C0088130000FFFFFF3FC3
:1052140070B5002849D00446064628367078002820
:1052240006D130701120C0026060204606F088F874
:10523400022070702068CA21416253214162C16812
:10524400490616D4C16880220A43C260FEF704F8F6
:1052540005462068C16849060BD4FDF7FDFF401BD5
:105264007D21C9008842F4D9032070702168CA687E
:1052740018E08169174A0A408261A16862690A4399
:10528400E169114382690A43826121690161E1682C
:10529400090402690A430261204600F01DF82168EE
:1052A400002804D0FF224A6270BD012070BD07208F
:1052B40040078A6982438A61206A626A0243A0695C
:1052C40010438A6902438A61FF204862012070709A
:0852D400002070BDBFFF8FFB3D
:1052DC00F0B581B00446234F38460C380168802263
:1052EC00914301607D20C6003868800615D4206883
:1052FC00C168A0229143C160FDF7AAFF0546206852
:10530C00C068800623D4FDF7A3FF401BB042F6D93A
:10531C0029210320605401B0F0BD38682021009190
:10532C00884338602068C168A0229143C160FDF7B2
:10533C008FFF05462068C06880060BD4FDF788FFF8
:10534C00401BB042F6D929210320605403E0002011
:10535C0001B0F0BD00203968009A1143396001B0EA
:08536C00F0BDC0461828004006
:10537400F0B583B004462820205C012802D1022025
:1053840003B0F0BD16460D46224628320220507066
:105394002068CA21416253214162012101911170A7
:1053A400C168490602921CD4C16880220A43C260C3
:1053B400FDF752FF07462068C168490611D4FDF77E
:1053C4004BFFC01B7D21C9008842F4D90320029FF2
:1053D40078702168CA68FF224A620021397003B0DC
:1053E400F0BD826940211140002E03D0002913D161
:1053F400E97013E0002900D1E9702A7800210A2A13
:1054040017D30A3AD3B2CD265E43F30A0A265E4383
:10541400921B1B0110330DE0E9788905029F019E60
:105424002A7812046B781B029A18AB78D3180B43B2
:105434002BE00B461343DAB213046A780A2A0AD320
:105444000A3AD6B2CD277743FE0A0A277743D21BFE
:105454003601103600E00E46029F1643F2B21202E5
:105464001A43AB780A2B09D30A3BD9B2CD264E4353
:10547400F10A0A264E439B1B09011031019E194370
:10548400C9B20A43E9788B0513430D4919400160F9
:10549400B10482698A438261E9682A690A4381699D
:1054A400114381612046FFF717FF2168FF224A62FA
:1054B400002892D17E700021397003B0F0BDC0463F
:0454C4007F7F7F0067
:1054C800F0B585B000280CD0044605465C3541206F
:1054D8008600606A002807D000202061204614302A
:1054E80007E0012005B0F0BD6068B04203D0204657
:1054F8001C30002101600027A7626878002803D1CA
:105508002870204606F02AF8022004950190687059
:10551800206801684022914303900160E168254AB0
:10552800012591422A4600D300221203ED020D43C1
:105538000F2738020290854201D00025A5626568D0
:10554800A768354021239B023B405B1925690198D8
:1055580005401D436069012318402843FC36A769AC
:105568003E400643E069382505403543206A8026D9
:1055780006402E435803A56A05403543039E35600F
:10558800380C04250540029801400A432A43606A02
:10559800102101401143606B082202400A437260E7
:1055A800D802F1698143F1610020206604994B70AB
:0855B80005B0F0BD0107000081
:1055C000F0B585B0044607464437387E012802D13D
:1055D000022005B0F0BD1D460292039101263E76E1
:1055E000FDF73CFE0490797E01297BD103980028C9
:1055F00000D14BE10298002800D147E1002D304650
:105600007CD0787E042801D005207876002323669C
:105610007D80E587E168A34A01200191914200D392
:105620001E46360302032068416891438919416090
:10563000029921643D800399A163E3642365A587F2
:105640000168490603D4016840220A4302600A9EA9
:1056500061684A424A41691E4B424B4113430199DA
:10566000904A91424ED3002B07D0039A1188C16013
:10567000901CA063E08F401EE087701C049B00D14B
:1056800084E0012505E0FDF7E9FD049BC01AB04266
:105690007AD2E08F002803D17888002800D1D2E0A8
:1056A0002068816889070DD5E18F00290AD0012D76
:1056B00008D1A16B0A88C260891CA163E18F491ED1
:1056C000E18700258168C907DDD079880029DAD013
:1056D000216CC0680880881C20647888401E78800F
:1056E0000125D0E74120820063680220934205D162
:1056F000A268002A02D1042900D177E70021397677
:1057000005B0F0BD002B08D0039909780173A06B98
:10571000401CA063E08F401EE087701C049B62D099
:10572000012505E0FDF79AFD049BC01AB0422BD27B
:10573000E08F002803D17888002800D183E020681A
:10574000816889070FD5E18F00290CD0012D0AD17E
:10575000A16B09780173A06B401CA063E08F401E11
:10576000E087206800258168C907DBD07988002997
:10577000D8D0007B216C0870206C401C2064788895
:10578000401E78800125CDE7032084E0012502E05A
:10579000FDF764FD049BE08F002802D17888002883
:1057A00051D02068816889070DD5E18F00290AD082
:1057B000012D08D1A16B0A88C260891CA163E18F09
:1057C000491EE18700258168C907E1D07988002951
:1057D000DED0216CC0680880881C20647888401E58
:1057E00078800125D4E7012502E0FDF737FD049B11
:1057F000E08F002802D17888002824D020688168B2
:1058000089070FD5E18F00290CD0012D0AD1A16B9A
:1058100009780173A06B401CA063E08F401EE087F5
:10582000206800258168C907DFD079880029DCD08D
:10583000007B216C0870206C401C20647888401E1E
:1058400078800125D1E703200490C102204632462A
:105850001D4600F029F800280FD1204631462A467F
:1058600000F0D4F8002808D10498410220463246BE
:105870002B4600F019F8002805D0206E202108439F
:10588000206621660120216E002904D0012000211C
:10589000397605B0F0BD012179760021397605B061
:0858A000F0BDC0460107000045
:1058A800F0B587B0049314460E46054605A80027B0
:1058B8000770FDF7CFFC0499081A02940419FDF744
:1058C800C9FC04904E48006823214143080D6043F9
:1058D800069003952D68A868304233D001970321BC
:1058E8004F020298401C30D0BE4200911CD104E007
:1058F800039800688068384245D0287B05A908705D
:105908000598FDF7A7FC0499401AA0423ED20698D4
:105918000699491E06910028EAD10024E8E7039871
:105928000068806830422ED0FDF794FC0499401A34
:10593800A0422BD206980699491E06910028EED15E
:105948000024ECE7002007B0F0BDBE4247D1287B19
:1059580005A908700598A868384214D0287B05A9BD
:1059680008700598A86838420DD0287B05A90870EA
:105978000598A868384206D0287B05A908700598BC
:10598800A8683842E3D1019807B0F0BD039C2068AD
:105998004168E022914341604121890062688A425E
:1059A8000BD1A1680122D303994202D092029142FD
:1059B80003D1016840229143016001214A03A36A8F
:1059C8005C34934205D1036893430360036813432F
:1059D8000360002020706170009807B0F0BD019945
:1059E800A868304208D0A868304205D0A86830427C
:1059F80002D0A8683042F3D1084607B0F0BDC046CF
:045A08002400002056
:105A0C00F0B583B015460F460446FDF721FC281A65
:105A1C00C519FDF71DFC06462C4800684001000D19
:105A2C0068430290226891680020090622D5791CEF
:105A3C001DD0019027465C3703E020688068000683
:105A4C0041D5FDF705FC801BA84215D2029802999E
:105A5C00491E02910028F0D10025EEE79168090655
:105A6C0008D59168090605D59168090602D5916893
:105A7C000906F3D403B0F0BD20684168E0229143DD
:105A8C0041604121890062688A420BD1A1680122E0
:105A9C00D303994202D09202914203D10168402271
:105AAC009143016001214A03A36A934205D1036823
:105ABC0093430360036813430360002038707970CC
:105ACC00032003B0F0BD019803B0F0BD240000200A
:105ADC00B0B5002823D0044605463C35687800282C
:105AEC0003D12870204608F0AFFC022068702068B3
:105AFC0003682E4A904202D02D49884211D1702160
:105B0C008B43A16819432B4B98420EDC284B9842CF
:105B1C0014D02C4B984211D090420FD043E001206E
:105B2C00B0BD1946234B9842F0DD234A904205D074
:105B3C00224A904202D0224A904234D103221202CD
:105B4C00914322690A4380218A43A1691143016070
:105B5C00E168C162616881621B494118890A82054A
:105B6C005118072906D801228A40E1210A4201D0A6
:105B7C006169016322463E3244340121416103696B
:105B8C00DB0702D003698B430361217111705170E3
:105B9C009170D1701171517121706170A170E170AF
:105BAC0069700020B0BD0A46CDE7C046002C01400C
:105BBC0000040040FF3F014000400140004801400C
:0C5BCC00004401400020004000D4FEBF57
:105BD80070B504463C340221617006463E360546DF
:105BE800443501680A6A0E4B1A4207D10A6A0D4BFE
:105BF8001A4203D10A6801239A430A6008F027FC75
:105C08000020287130707070B070F0703071707151
:105C180028706870A870E8702070607070BDC04609
:085C280011110000440400000A
:105C3000F0B581B004463E340346443301270029C1
:105C400018D000908D070E1FB608A81903283BD85E
:105C5000860001A7BE59B746695C00089B5C000836
:105C6000A75C0008B35C0008661C3678012508298B
:105C700024D12EE022781D786D1E6E1EB541012ABA
:105C80003E4600D12E46002E2FD1022222701A70DD
:105C90000B46D341032B28D863E0A61C3678012598
:105CA00008290BD115E0E61C36780125082905D115
:105CB0000FE0261D3678012508290AD0042901D1D4
:105CC0005F1C07E0DF1C05E0661D3678012508290A
:105CD000F4D19F1C3F787F1E7A1E9741012E2E46DD
:105CE00000D13E46002E03D00127384601B0F0BD5A
:105CF00003282F460CD8C0467844007940008744DA
:105D0000010D1326022262700098082911D123E0A8
:105D100002226271009808290BD11DE00222A270B4
:105D20000098082905D117E00222E270009808299E
:105D300012D0042905D15A700B46D341032BD4D875
:105D40000FE0DA700B46D341032BCED809E00222D4
:105D5000227100980829ECD19A700B46D341032B8D
:105D6000C3D89A00144B9B580268D0681843D0607F
:105D70001F200140012318468840116A81431162A7
:105D8000116A014311620D48824205D00C488242DB
:105D900002D00C48824208D190680B49014000278C
:105DA0000629A2D0180481429FD0106818431060C1
:105DB000002001B0F0BDC046F8DD0008000400403E
:0C5DC00000400140002C014007000100E1
:105DCC0030B502230A46DA41032A31D89200284B17
:105DDC009A580368DC681440DC601F240C400122D4
:105DEC001546A5401C6AAC431C621C6A1C621C6AEA
:105DFC00204D2C4206D11C6A1F4D2C4202D11C682E
:105E0C0094431C6003463E334430002912D08C0767
:105E1C000D1FAD086419032C10D8C0467C4424799E
:105E2C006400A744010F131E5A70082911D11BE0FE
:105E3C00012030BD1A700270002030BD5A71082943
:105E4C0007D111E09A70082903D10DE0DA70082906
:105E5C000AD0042902D14270002030BDC27000204B
:105E6C0030BD1A710829F4D18270002030BDC046B3
:0C5E7C0008DE00081111000044040000C2
:105E8800F0B583B004460068C56802272946394042
:105E98004A424A410169029139404B424B411343FE
:105EA80013D16A49FE310161012121778069800798
:105EB80003D0204600F0FAFE05E0204608F0C8FAB4
:105EC800204608F0C6FA0020207701260422294639
:105ED80011404842484102994907314600D50146D8
:105EE800032000020190002916D10092206857492A
:105EF800FC310161277780690199084203D0204667
:105F080000F0D4FE05E0204608F0A2FA204608F08A
:105F1800A0FA00202077009A0827294639404842ED
:105F2800484102990907314600D50146002913D195
:105F380020684649F83101612277C069800703D09B
:105F4800204600F0B3FE05E0204608F081FA20461E
:105F580008F07FFA00202077102129404842484164
:105F68000299C906314600D50146002914D1206896
:105F78003649F03101612777C0690199084203D099
:105F8800204600F093FE05E0204608F061FA20461E
:105F980008F05FFA00202077012129404842484153
:105FA8000299C907314600D00146002906D1206868
:105FB8002649FF310161204608F04CFA80272F401E
:105FC800784278414121C901029A0A42314600D0FB
:105FD8000146002905D120681D490161204608F0C5
:105FE8003CFA784278410299C905314600D5014604
:105FF800002905D1206815490161204608F02EFACC
:10600800402129404842484102994906314600D575
:106018000146002906D120680C49C031016120469B
:1060280008F019FA2020054068426841029989065B
:1060380001D403B0F0BD0600FBD120680349E0316C
:106048000161204608F008FA03B0F0BDFFFEFFFF2B
:046058007FDFFFFFE8
:10605C00F0B582B03C23C35C012B02D1022002B00C
:10606C00F0BD03463C330224E241032A00D9A4E0EC
:10607C007A44127952009744012E52730268146AC2
:10608C00156A012085431562CD68019560C900969B
:10609C0097694D4E0839B24205D04C4EB24202D0EF
:1060AC004B4EB24202D1032087430098074310465F
:1060BC001830F026B743019E3601F6B2BE19966130
:1060CC000A263540B4436419146294690C25AC4318
:1060DC009461896869E00068026A046A1025AC431F
:1060EC0004624C682402374D2540CC682403A4B2CA
:1060FC006419F3252D028669AE43264386610C682C
:10610C002401A0252C40AA431219026203229202F8
:10611C0084699443846189680902183045E00068F9
:10612C00026A01242402056AA54305624C68F02525
:10613C00AC43CD682D01EDB22C19C569F326B543DE
:10614C002543C561052464020D682D022540A24338
:10615C0052190262C2690C24A243C261896823E00D
:10616C000068026A01242403056AA54305624C6891
:10617C002402144D2540CC682403A4B26419F325E1
:10618C002D02C669AE432643C661052464030D681F
:10619C002D032540A2435219026203229202C469C4
:1061AC009443C461896809021C3002680A43026086
:1061BC0000200021197002B0F0BD012000211970DF
:1061CC0002B0F0BD000FFFFF000400400040014092
:0461DC00002C014052
:1061E0000222D141032909D87944097949008F4411
:1061F00001070B0F006834300068704700207047BB
:10620000006838300068704700683C3000687047AC
:0862100000684030006870478F
:1062180010B53C23C35C012B01D1022010BD0346FD
:106228003C33002A05D0082A06D0042A0ED10A4A8F
:1062380003E00F22D24300E0064A0068846E14404F
:106248000C43846600200021197010BD0120002134
:0C625800197010BDFFFFF0FFFFF0FFFF0A
:1062640070B50446026810686F490140A06823694C
:10627400034360691843636E03430B43E1690B43B3
:1062840013600320000353688343E068184350609D
:10629400A069236A03439068644D05401D439560DB
:1062A400D36A0F208343606A0343D3620023604DA3
:1062B400AA4206DC614DAA4212D0614DAA4215D011
:1062C4000CE05C4DAA4211D05B4B9A4206D15D4A68
:1062D40012689207120F5C4B9B5807E0102305E0ED
:1062E400584A12680C231340574AD3582646683636
:1062F4000125EA03914215D1082B00D98DE0C0464F
:106304007B441B795B009F44048823882988888800
:106314003300FEF7ADFE626A0B2A24D291004C4A88
:10632400515846E0082B00D977E0C0467B441B79DE
:106334005B009F4404722372297272723300FEF769
:1063440097FE626A0B2A24D29100414A515857E0C1
:106354000B2829D280003E49095829E0FEF744FE63
:10636400626A0B2ADAD301210B2A22D1090220E026
:106374000B2824D240003549095A24E00B2833D293
:1063840080003349095833E0FEF72EFE626A0B2A77
:10639400DAD301210B2A33D1090231E00B2829D2A7
:1063A40040002A49095A29E001210B2800D1090299
:1063B400284806F067FC400061684A080AE00121A9
:1063C4000B2800D109020120C00306F05BFC420047
:1063D40061684808101806F055FC1F4901401CD09C
:1063E4000007400F084315E001210B2800D10902E2
:1063F400184805E001210B2800D109020120C0033F
:1064040006F040FC61684A08101806F03BFC80B2B4
:10641400102802D32168C86000251048306000208D
:10642400E0662067284670BDF369FFCFFFF4FF11D3
:10643400FF4B0040004C0040003801400044004045
:10644400004800405410024018DE000822EA000808
:1064540028DE00080024F400F0FF00000100010021
:10646400F0B581B0044606467C3600200090F0600A
:10647400FCF7F2FE05462168086800070ED5C869D6
:1064840080020BD401204705FCF7E6FE401B21687F
:10649400174A90421AD8C8693842F5D008684007AC
:1064A400009A10461DD5C8694002104619D401202F
:1064B4008705FCF7D1FE401B21680D4A904205D8A0
:1064C400C8693842F5D0009A10460AE00D20400110
:1064D4000A6882430A608868012290438860032026
:1064E400009A202171603270B16001B0F0BDC046E5
:0464F400FFFFFF01A6
:1064F800F0B581B004467C3465680223202D12D1A2
:10650800012500290CD0002A0AD0866800952F039F
:10651800BE420BD1CD0709D00569002D06D1009DDB
:10652800284601B0F0BD022001B0F0BD2578012D4C
:106538001D46F5D0034654335A800025E5601A807D
:10654800016521216160009B5907426E8A4206D18C
:10655800BE4202D10169002908D0114907E0BE42B4
:1065680002D10169002909D00B4908E00B49002232
:1065780022700167D9050068083004E005492570D4
:1065880001670068802102680A430260002001B0A8
:10659800F0BDC046096600088BE50008AD65000837
:0465A80039E50008C9
:1065AC0070B58021415821291AD102465632938A5E
:1065BC00002B15D00168104C02E05B1E1D040FD09F
:1065CC001588002D0DD0CD692D06F6D5056D2E88BC
:1065DC0026408E62AD1C056515886D1E1580ECE796
:1065EC0070BD0120C0058A6882438A600868402219
:0C65FC0002430A6070BDC046FF010000B1
:1066080010B58022815821290FD1014656310B88B7
:10661800002B0BD0026D1388094C1C4003689C6248
:10662800921C02650888401E088010BD0068016839
:1066380091430160016840220A43026010BDC046D0
:04664800FF0100004E
:10664C00F0B584B004467C34A3680227202B13D108
:10665C00012300290DD0002A0BD0866801252B03BD
:10666C0003939E420BD1CB0709D00369002B06D1B3
:10667C000123184604B0F0BD022004B0F0BD23780D
:10668C00012B3B46F5D003465C335A801A8081655A
:10669C00002E00930AD029078E420CD003998E420B
:1066AC000ED10169002904D126490CE001690029A9
:1066BC0008D1FF2107E00169002903D03F2102E046
:1066CC00002100E07F2199800023E3602221A1605A
:1066DC000768B96829430197B960290202916907D3
:1066EC00476E8F4203D10099898991420ED9039943
:1066FC008E4202D10169002910D0164A029D019EDA
:10670C0000212170C2662035324615E003998E4275
:10671C0002D10169002903D00C4E02E00C4AEDE7CE
:10672C00094E019F3A46083200212170C66638682E
:10673C000299084338602D07106828431060002028
:10674C0004B0F0BDFF010000656700080568000893
:08675C00C5E500081FE6000876
:10676400F0B581B004468420205822282BD1254638
:106774005E356E89002E2AD02046843000906F88C2
:1067840002E0761E300422D02068416A3940A26DAE
:1067940011802988491E2980911CA1652988002916
:1067A400EFD10121090202688A4302608168124A1A
:1067B400114081600020E066202000990860204696
:1067C40007F05BFFDDE72068183008210EE0288819
:1067D40000280ED0698988420BD20848E066064832
:1067E400411C206882680A408260202102680A43B2
:1067F400026001B0F0BDC046FEFFFFEFC5E5000832
:10680400F0B581B004468420205822282DD1254695
:106814005E356E89002E2CD02046843000906F881F
:1068240002E0761E300424D02068406A3840A16D0E
:1068340008702888401E2880A06D401CA065288808
:106844000028EED10120000221680A6882430A6010
:106854008868124A104088600020E0662020009971
:106864000860204607F009FFDBE72068183008219C
:106874000EE0288800280ED0698988420BD2084887
:10688400E0660648411C206882680A408260202134
:1068940002680A43026001B0F0BDC046FEFFFFEF8C
:0468A4001FE60008E3
:1068A800F0B581B000249A4D2346009406E00546D1
:1068B8004354002B7BD05B1C802B7FD0284699004B
:1068C800924A555820328027214603E0103F403233
:1068D800002FECD01646203E3668B54200DD491C34
:1068E80016461C3E3668B54200DD491C1646183E61
:1068F8003668B54200DD491C1646143E3668B54276
:1069080000DD491C1646103E3668B54200DD491CBC
:1069180016460C3E3668B54200DD491C1646083E50
:106928003668B5421CDC161F3668B5421DDC166891
:10693800B5421EDC5668B5421FDC9668B54220DCBD
:10694800D668B54221DC1669B54222DC5669B542E3
:1069580023DC9669B54224DCD669B542B6DD24E06D
:10696800491C161F3668B542E1DD491C1668B54258
:10697800E0DD491C5668B542DFDD491C9668B54222
:10698800DEDD491CD668B542DDDD491C1669B54215
:10699800DCDD491C5669B542DBDD491C9669B54208
:1069A800DADD491CD669B54290DD491C8EE70098AE
:1069B800012800D1A6E0012300937FE75549402430
:1069C8000C70002203E01032802A00D198E0A85C05
:1069D80084422ED0AB185878844230D098788442BC
:1069E80033D0D878844236D01879844239D058794F
:1069F80084423CD0987984423FD0D879844242D0AE
:106A0800187A844245D0587A844249D0987A844288
:106A18004DD0D87A844251D0187B844255D0587BC7
:106A2800844259D0987B84425DD0D87B8442CAD1B5
:106A380061E00A70D4B2AB1858788442CED1501CA9
:106A48000870C4B298788442CBD1901C0870C4B244
:106A5800D8788442C8D1D01C0870C4B2187984424E
:106A6800C5D1101D0870C4B258798442C2D1501DD6
:106A78000870C4B298798442BFD1901D0870C4B21E
:106A8800D8798442BCD1D01D0870C4B2187A844227
:106A9800B9D1104608300870C4B2587A8442B5D1CA
:106AA800104609300870C4B2987A8442B1D11046B1
:106AB8000A300870C4B2D87A8442ADD110460B307F
:106AC8000870C4B2187B8442A9D110460C300870F3
:106AD800C4B2587B8442A5D110460D300870C4B2A8
:106AE800987B8442A1D110460E300870C4B2D87B7E
:106AF800844200D067E710460F300870C4B262E7DE
:106B080001B0F0BD044806F087F9FEE7FC07002055
:0C6B1800CA1300202900002068EC0008CF
:106B240080B500F07FF802480421016080BDC046B2
:046B3400A80F002086
:106B3800F0B583B000F074F8314F0420029038604B
:106B48003048006800900023304C07E00026019B85
:106B5800980032490E505B1C802B45D0294A10689A
:106B68002949084001931902014311600BE00120F3
:106B7800386000212046FFF757F81520FDF74EF939
:106B88000226022EE3D138680428F0D0386802269D
:106B98000328F6D138680328D8D11520FDF74AF91B
:106BA800002520462946FFF70DF902983860184855
:106BB8000168002908D0174B1868174A1268120391
:106BC80080181860092903D8481C11490860D8E7BB
:106BD8000F490D600F490D600A2106F051F8216830
:106BE800896A4E1C4643CCE77F200002009A024087
:106BF80004490868044B18401043086003B0F0BD0E
:106C0800A80F002004100240FF80FFFF540E002050
:106C1800480F00205C0F0020AC0F0020FC0700206C
:106C280070B584B0012670041C490A6802430A60E2
:106C38001B4D1C4A2A6009680140009100982846AB
:106C4800FEF7C6FF184800246C60AC60E8602C6151
:106C58002846FEF73FFF002800D0FEE703940C20EB
:106C68000290019600940E4869460022FFF7F2F957
:106C7800002800D0FEE70A4802210022FFF7C8FAE0
:106C8800002800D0FEE7152000210A46FDF7AAF8E3
:106C98001520FDF7CFF804B070BDC0464010024083
:0C6CA800540E002000440140FFFF0000DB
:106CB400F0B581B00446007F01283CD11F4E3068F6
:106CC400012807D100212046FFF788FA1E490860F1
:106CD40002202FE0306802282DD100212046FFF742
:106CE4007DFA174F38601520FDF7A6F815480021E6
:106CF400FFF76AF80220C04321680861124800685F
:106D04003968814201D9081A03E0FED2081A0F49F2
:106D140040180F490860086800030E49884208D2E9
:106D24000D4806F07BF80A48006801030B4806F09A
:106D340075F80320306001B0F0BDC046A80F0020F4
:106D4400940F0020540E0020980F0020FFFF000035
:106D5400AC0F0020405DC600D9F00008EAF000083E
:106D6400F0B583B00D46029001600C20454906C57C
:106D74000021E86029616961A961E961296201264C
:106D84003703083D2C467C340998089A002B04D01C
:106D9400012B04D10321490202E0B10200E00F46B5
:106DA400AF602961511E4A1E91414903E96005F013
:106DB400DFFE0027344B3A4607F09DFC05F050FEF9
:106DC40001906068002803D12770284604F0D4FCA1
:106DD4002420606028680168B14301602846FFF7F9
:106DE4003FFA012835D0A86A002802D0284607F0C7
:106DF40038FBB0032C68A1680143A160F003A168CB
:106E04008143A1602068214901402160F005616847
:106E140001436160B0062168014321606F6803206B
:106E24004002D63078431A4905F02CFF19498F42A5
:106E3400019A00D3421CFF200006616901401143FE
:106E440061612068304320602846FFF709FB002871
:106E540001D007F02EFC029C206807F00FFC0028EC
:106E640001D007F026FC2068273432022146FFF7C0
:106E7400EBFB002803D0084805F0D0FFFEE703B081
:106E8400F0BDC0460038014000000C40FFFF00FC8C
:0C6E940040420F00014B00006BEE0008B4
:106EA000F0B58DB005460268D16910680C90506845
:106EB00001200A90000709900695803590680B9094
:106EC0000807089049D00998431C0B9803400126F5
:106ED00037023C4620340C9804401C433DD0074008
:106EE0007C427C41CF070A9F00D02746002F03D168
:106EF0001662AC683443AC600B980640744274412F
:106F00008F070A98074600D52746002F05D102248F
:106F10001462AC6804272743AF60744274414E0783
:106F2000064605D4002E05D0089800280BD414E09E
:106F30002600F9D104241462AC6802262643AE6010
:106F40000898002809D520240C9804401C4304D03C
:106F500008231362AC681C43AC600126F00507905F
:106F60000B050FD50B9B0340B4060C980440E318A7
:106F700008D0F302136220236B602B60624B1E75F6
:106F8000624C1E55059620200F460890074022D0DF
:106F90000B9B099803400C9C089804401C431AD092
:106FA0006B68222B13D14523DB005748C658059840
:106FB0000402A6420BD2544CA019526A27268255CD
:106FC000524A0598A054E258521CE25003E09369DB
:106FD00008241C43946180240E4626400A98049499
:106FE00039D00B9A079B1A400C9B2340134332D095
:106FF000454A136822461C59212C039713D11C467D
:1070000056342288002A17D01A6802921A6D01920B
:1070100012782746029CA262019A521C1A653A888D
:10702000521E3A8011E01F683B6893433B603B6807
:1070300040241C433C6008E01A681368049FBB436B
:107040001360136840241C43146023221201059B23
:107050002D4FBB54039F40240C9B23405A425A415E
:10706000490606D4002806D0A868002815D10DB01E
:10707000F0BD1000F8D12648002101700698036881
:107080001A68A2431A6001670899296007F0F6FAA6
:1070900022206860A8680028E9D022236B60002FB6
:1070A00007D00B98099901400C98089A10400843A2
:1070B0001FD1002EDBD00B99079801400C98049A41
:1070C00010400843D3D026200F4E0021315406989B
:1070D000222703681A68A2431A6001670899296089
:1070E00007F0CCFA6F6023200001059931540DB0F0
:1070F000F0BD06980068816908220A438261002079
:10710000A8600DB0F0BDC046C805002031020000E7
:04711000EE05002068
:10711400F0B585B04521CD004159052900D2BBE029
:1071240003952722825C00920346273301220C46F2
:1071340014400494D5438A1E0192154002935B1CAB
:10714400674A684E03E0AD1E9B1C002D71D05C1E87
:10715400247854406208E40730D15708D20731D16B
:107164007A08FC0732D15708D20733D17A08FC07D2
:1071740034D15708D20735D17C08FA0736D16208D2
:10718400E40700D072401C7854406208E40732D10E
:107194005408D20733D16208E40734D15408D20723
:1071A40035D16208E40736D15408D20737D16708CD
:1071B400E20738D17A08FC07C5D038E07240570896
:1071C400D207CDD077407A08FC07CCD0724057085C
:1071D400D207CBD077407A08FC07CAD07240570850
:1071E400D207C9D077407C08FA07C8D07440620837
:1071F400E407C7D1C7E772405408D207CBD0744024
:107204006208E407CAD072405408D207C9D0744057
:107214006208E407C8D072405408D207C7D074404B
:107224006708E207C6D077407A08FC078BD0724023
:1072340089E7049C002C1BD05B1E1B785A40530822
:10724400D20730D15A08DB0731D15308D20732D1E3
:107254005A08DB0733D15308D20734D15A08DB0765
:1072640035D15308D20736D15A08DB0700D0724013
:1072740001AB38CBE35C0C19641E24782402E318B8
:10728400934209D1491C07D00221009B002B07D04F
:10729400154A128B9A4203D04219002101751160DC
:1072A400084605B0F0BD73405A08DB07CDD07240E4
:1072B4005308D207CCD073405A08DB07CBD07240B6
:1072C4005308D207CAD073405A08DB07C9D07240AA
:1072D4005308D207C8D073405A08DB07C7D1C7E7A1
:0C72E400FFFF000001A0000030000020AF
:1072F000F0B585B0054627202B5CFF2420462830BA
:107300002B544521C9006918002702914F602818A5
:107310002946273101260490324600F0E5F803465D
:107320000395263501950028204600D1A7E0184690
:10733000304000906A4A6B4D012B05D13C463846DF
:10734000009900297ED19AE01846B043049E03E0DC
:10735000B61CBF1CB84270D0317869404C08C907D0
:1073600030D16508E10731D16C08E90732D16508F1
:10737000E10733D16C08E90734D16508E10735D15D
:107380006908EC0736D14C08C90700D0544075781D
:1073900065406908EC0732D14C08C90733D1610850
:1073A000E40734D14C08C90735D16108E40736D168
:1073B0004C08C90737D16108E40738D14D08C9071F
:1073C000C6D038E054406508E107CDD055406C0880
:1073D000E907CCD054406508E107CBD055406C0894
:1073E000E907CAD054406508E107C9D0554069088B
:1073F000EC07C8D051404C08C907C7D1C7E7514076
:107400004C08C907CBD054406108E407CAD05140AA
:107410004C08C907C9D054406108E407C8D051409E
:107420004C08C907C7D054406108E407C6D0514092
:107430004D08C9078CD055408AE7280A2C46009988
:1074400000291CD00498C05D45406808E9072AD18E
:107450004108C0072BD14808C9072CD14108C007F3
:107460002DD14808C9072ED14108C0072FD148089F
:10747000C90730D14408C00700D05440200A0499FD
:10748000CC54CA1850700C20019A10709A1C029D9E
:107490006A60039C206892B2FFF72EF800202860F3
:1074A000207505B0F0BD50404108C007D3D0514011
:1074B0004808C907D2D050404108C007D1D0514038
:1074C0004808C907D0D050404108C007CFD051402C
:1074D0004808C907CED050404408C007CDD1CDE7F9
:0874E00001A00000FFFF000005
:1074E800F0B586B04C78102C11D0062C1DD0032C8A
:1074F8002AD1914C258B002B2FD09D422DD086214F
:107508008154551C0B214155901C06B0F0BD0590C7
:107518008948048B022601200490002B2FD09C421E
:107528002DD00B2586241346A9E0834C258B002BF0
:1075380035D09D4233D086218154531C02240B211F
:10754800C154A01806B0F0BD80214C408454801866
:1075580001214170901C06B0F0BD4E790B791B02D9
:107568009B191D467E3D7D27FF43BD4227D88321B9
:107578008154551C03214155901C06B0F0BD487933
:107588000B791B021B181C467C3C7A25ED4390277F
:107598000397AC4228D20325134690246FE0059048
:1075A800CD788B781E027619B708772F6FD386218E
:1075B8008154531C0221C154881806B0F0BDCD78FF
:1075C800897804910902039549195B185B4D5D1987
:1075D8006F1E551C594CA74270D283218154022139
:1075E8004155901C06B0F0BD0090C87801908C7889
:1075F800029424022718D819504BC5186E1E02256C
:107608009E4213462E46039C39D30392019A530097
:10761800029A5502EB18484AD318049300250246EB
:10762800184646194B19DC7974701C7A44557C1C31
:10763800944215D25C7AF4709C7AB470BC1C944263
:107648000ED2DC7A74711C7B3471FC1C944207D214
:107658005C7BF4719B7BB37108353F1D9742E0D387
:1076680010200599039A8854881801998170029905
:107678004170D31C0526042004900024009D059920
:10768800CC54049880180D54B01806B0F0BD7000A2
:10769800271804970F79049E77704F79275406248A
:1076A800059884548418A57063700B79E370131DD2
:1076B80049790524C154A01806B0F0BD03278754A2
:1076C80076004655801805900398450004984602B0
:1076D8007519194845190024059806192F1978783D
:1076E800B070285DF070481C984219D2F878307153
:1076F800B8787071881C984216D27879B071387948
:10770800F071C81C984213D2F8793072B879707247
:107718000834091D9942DFD31019801C06B0F0BD4A
:107728001019001D06B0F0BD1019801D06B0F0BD7F
:107738001019083006B0F0BD3000002024FEFFFF0D
:10774800F0B583B03C214848012747542C214754C1
:1077580000240C25056444648464C464072181639F
:107768004163446284620826C661877604833F4980
:107778003A030263021D1477016079050322920718
:1077880042608460C460016146610294019400947F
:10779800FBF778FD002801D006F089FF02940194D8
:1077A800009731486946FBF787FF002801D006F0AB
:1077B8007EFF0294042001902D4800902A486946D3
:1077C800FBF77AFF002801D006F071FF02940196BA
:1077D8002848009024486946FBF76EFF002801D02E
:1077E80006F065FF02940195234800901E486946FB
:1077F800FBF762FF002801D006F059FF0294102021
:1078080001901E48009018486946FBF755FF00286C
:1078180001D006F04CFF0294142001901848009003
:1078280011486946FBF748FF002801D006F03FFFE2
:10783800029418200190134800900B486946FBF702
:107848003BFF002801D006F032FF02941C20019073
:107858000D48009004486946FBF72EFF002801D028
:1078680006F025FF03B0F0BD940D00200024014070
:1078780002000004040000080800000C10000010BA
:0C7888000001002000040028001000B0E7
:10789400F0B58BB000240A940994026845498A42E1
:1078A40001D00BB0F0BD0290012319054248C26813
:1078B4000A43C260C2680A400592059901681943E7
:1078C4000160016819400493059105990168022239
:1078D40003921143016000681040059005980894D4
:1078E40003270797069305200190050706AE28464F
:1078F4003146FCF72DFF0894079703980690284615
:107904003146FCF725FF0894079704200090069061
:1079140028463146FCF71CFF089407970498069004
:1079240026483146FCF714FF0894079703980690FD
:1079340022483146FCF70CFF0894079700980690FC
:107944001E483146FCF704FF089407970820069068
:1079540028463146FCF7FCFE089407971020069051
:1079640028463146FCF7F4FE154D2C622020049A7B
:10797400D10212028023134E2E60019E6E60AC6011
:10798400EC602B616A61A961E8612846FCF7BAFAE8
:10799400002801D006F08DFE0298A86205650C202F
:1079A40000210A46FCF720FA0C20FCF739FA0BB048
:1079B400F0BDC046002401403410024000040050D1
:0879C400F80D0020080002404C
:1079CC00F0B589B007910646049008AD22200390CB
:1079DC0028700520070701200190C403002206929D
:1079EC003846214607F060F80A20059000900323E2
:1079FC000293304629462A46FDF7DCFD38462146DF
:107A0C00019E324607F050F842202870A8780721D2
:107A1C00014007980143697038462146069A07F0E1
:107A2C0043F8059800900223049829462A46FDF74E
:107A3C00C1FD38462146324607F036F803982870C7
:107A4C0038462146069A07F02FF8059800900498BE
:107A5C0029462A46029BFDF7ADFD384621463246A3
:107A6C0007F022F8A87807990840884201D109B09C
:107A7C00F0BD024805F0CEF9FEE7C046E0F2000882
:107A8C0080B53121C900415881670146CC314A8803
:107A9C007C23C252CC22825A7C304280896841605D
:107AAC000248002102F0CAFA80BDC0463000002016
:107ABC0010B504468034616D616061688022805825
:107ACC00091A7D20C20005480068504305F0AEF845
:107ADC00A0600348002102F0B1FA10BD6C0F002029
:047AEC003000002046
:107AF00010B5CC200A4C205A8C216052605E7E2149
:107B0000615E411A7D20C20006480068504305F0BE
:107B100093F8902160500021204602F095FA10BDA4
:087B200030000020740F00206A
:107B2800F0B581B00546324805F076F99435A86875
:107B3800002858D0A86804F0CDFF2E4B002204F08E
:107B480029FE2D4AC0CA32463B4604F023FE2B4B81
:107B5800002206F0CEFD04F01BFF2860688FA88085
:107B6800288FE880264832463B4605F055F9A86834
:107B780004F0B0FF00221F4B04F00CFE024621481F
:107B88000B4605F049F90420285E04F0A3FF1E4EB9
:107B98000022334604F0FEFD02461C480B4605F061
:107BA8003BF90620285E04F095FF0022334604F0D6
:107BB800F1FD024616480B4605F02EF9286804F038
:107BC80089FF00220D4B06F094FD024611480B4632
:107BD80005F022F9104805F01FF91048002102F0BD
:107BE8002FFA01B0F0BD0E4805F016F901B0F0BD4E
:107BF80079EE000800408F40A005002080842E41C7
:107C080003F100087FEC0008000059408EEC0008E2
:107C1800E5EE0008FCF20008EFEE00083000002056
:047C28008BEE0008D7
:107C2C00F0B583B03A4805F0F5F8CE24394F385BFF
:107C3C00A0217852785E04F04BFF374E0022334679
:107C4C0004F0A6FD024635480B4605F0E3F8385F14
:107C5C009821795E3C46401A04F03AFF029001915B
:107C6C000022334604F094FD02462D480B4605F0E5
:107C7C00D1F82C480668436800932B48324605F02F
:107C8C00C9F89C27E05904F023FF284B002204F08C
:107C9C007FFD024626480B4605F0BCF8E059274606
:107CAC0004F016FF0022214B04F072FD3246009BBB
:107CBC0004F06EFD1F4B002204F022FC029A019B83
:107CCC0004F066FD1C4C0022234606F010FD04F067
:107CDC005DFEA4217850785804F0FAFE0022234669
:107CEC0004F056FD00220C4B06F001FD134B002254
:107CFC0004F006FC024612480B4605F08BF81148BE
:107D0C0005F088F83846002102F098F903B0F0BD70
:107D1C0099EC00083000002000005940B0EC00083D
:107D2C0005EF000890050020BFEC000800408F40D4
:107D3C0013EF00080000F0BF65CDCD410000F03F0F
:087D4C00F2EC000810F300083E
:107D5400F0B58FB0052004070122099211030791A1
:107D6400204606F0A5FE9620FBF77CFA80481021F9
:107D74000026324606F09CFE9620FBF773FA7C48F8
:107D84001021099A06F094FE9620FBF76BFA202145
:107D94007748324606F08CFE9620FBF763FA744867
:107DA4002021099D2A4606F083FE9620FBF75AFA05
:107DB40020460799324606F07BFE072002210691F1
:107DC4003246FCF711F80720FCF72AF80DAF3246CB
:107DD4000596BE70674838802E46ED032046294636
:107DE40006F066FE0A200A900090634839463A4637
:107DF400069BFDF7E3FB20462946324606F058FE73
:107E04002620387020462946059A0A9E06F050FE20
:107E140000960323584839463A46FDF7CFFB2046DF
:107E240008952946099A06F043FEB8780A2800D036
:107E340099E09620FBF716FA4F482021FFF7C4FD7E
:107E44000DAD232006902870002209922046089F39
:107E5400394606F02DFE009603230493464829462E
:107E64002A46FDF7ABFB012205922046394606F06F
:107E74001FFE432002902870A878EF21014069700A
:107E840020463946099E324606F012FE0A980090B2
:107E940002230393384829462A46FDF78FFB2046E0
:107EA4003946059A06F004FE06982870204639469D
:107EB400324606F0FDFD0A9800902F4829462A46CE
:107EC400049E3346FDF77AFB20463946059A06F0B0
:107ED400EFFD0DAD0698287020463946099A06F044
:107EE400E7FD0A980090244829462A463346FDF7C0
:107EF40065FB20463946059E324606F0D9FD0298B8
:107F04002870A8789F2101402031697020463946A5
:107F1400099A06F0CDFD0A980090174829462A468A
:107F2400039BFDF74BFB20463946324606F0C0FD65
:107F34000698287020463946099A06F0B9FD0A9831
:107F440000900D4829462A46049BFDF737FB20463E
:107F54003946324606F0ACFDA878800612D40748AC
:107F640004F05CFFFEE7064804F058FFFEE7C04655
:107F740000040050460A0000300D00202CF30008D5
:107F840020F100080DAD099EAE70342068705120B8
:107F9400287020463946324606F08AFD0A98009039
:107FA4001148022329462A46FDF708FB01220692BE
:107FB4002046394606F07CFD31202870204639469B
:107FC400324606F075FD0A980090032306482946B8
:107FD4002A46FDF7F3FA20463946069A06F068FD6C
:107FE400A878342808D001E0300D0020014804F0BE
:107FF40015FF01E015ED00080DAE099AB2700D48A9
:1080040030800BADAA702A802046394606F050FD18
:108014000A9800900848032331462A46FDF7CEFA11
:1080240001222046394606F043FD2878FF280CD16A
:1080340004E0C04625EC0000300D00200DA80078B7
:108044000BA94978814200D1A2E00DAE099AB27021
:108054000C4830800BADAA702A802046394606F0C1
:1080640027FD0A9800900848032331462A46FDF765
:10807400A5FA01222046394606F01AFD2878FF2881
:108084000AD103E025EC0000300D00200DA8007893
:108094000BA9497881427BD00DAE099AB2700D4884
:1080A40030800BADAA702A802046394606F000FDC8
:1080B4000A9800900848032331462A46FDF77EFAC1
:1080C40001222046394606F0F3FC2878FF280BD11C
:1080D40004E0C04625EC0000300D00200DA8007817
:1080E4000BA94978814253D00DAE099AB2700D485C
:1080F40030800BADAA702A802046394606F0D8FCA1
:108104000A9800900848032331462A46FDF756FA98
:1081140001222046394606F0CBFC2878FF280BD1F3
:1081240004E0C04625EC0000300D00200DA80078C6
:108134000BA9497881422BD00DAE099AB2700E4832
:1081440030800BADAA702A802046394606F0B0FC78
:108154000A9800900948032331462A46FDF72EFA6F
:10816400012620463946324606F0A2FC2878FF282C
:1081740006D000F0FFFCC04625EC0000300D0020C6
:108184000DA800780BA94978814201D000F0F2FCD7
:108194000BA8099A81786020049001430DAE0691E2
:1081A40071704520059030700BAD2A802046394609
:1081B40006F07EFC0A9800900748022331462A46BE
:1081C400FDF7FCF901222046394606F071FC2878B7
:1081D400FF280AD102E0C046300D00200DA8007827
:1081E4000BA94978814200D19AE00DAE06987070CF
:1081F400059830700BAD099A2A802046394606F05E
:1082040057FC0A9800900748022331462A46FDF796
:10821400D5F901222046394606F04AFC2878FF2881
:1082240008D101E0300D00200DA800780BA9497891
:10823400814275D00DAE06987070059830700BAD04
:10824400099A2A802046394606F032FC0A980090A2
:108254000748022331462A46FDF7B0F90122204699
:10826400394606F025FC2878FF2809D102E0C046EB
:10827400300D00200DA800780BA9497881424FD019
:108284000DAE06987070059830700BAD099A2A806F
:108294002046394606F00CFC0A9800900748022351
:1082A40031462A46FDF78AF901222046394606F06E
:1082B400FFFB2878FF2809D102E0C046300D0020DA
:1082C4000DA800780BA94978814229D00DAE0698F3
:1082D4007070059830700BAD099A2A802046394693
:1082E40006F0E6FB0A9800900848022331462A4625
:1082F400FDF764F9012620463946324606F0D8FBDC
:108304002878FF2804D000F045FCC046300D00203A
:108314000DA800780BA94978814201D000F03AFCFD
:108324000DAD099FAF8011480D90114802222946D6
:1083340005F092FEA8700BAEB7800B972046089903
:108344003A4606F0B5FB0A9800900A4806232946E7
:108354003246FDF733F901222046089906F0A8FBBE
:10836400301D06903078FF282BD105E025EC000065
:10837400CC0E0020300D00200DA800780BA9497800
:1083840081421ED10DA840780BA98978814218D169
:108394000DA880780BA9C978814212D10BA8457920
:1083A40003480122069905F057FEA84209D101E0CD
:1083B400CC0E00200BA8007904990840602800D155
:1083C4003BE10DADAF8010480D90104802222946C4
:1083D40005F042FEA8700BAEB7800B9720460899B3
:1083E4003A4606F065FB0A98009009480623294698
:1083F4003246FDF7E3F801222046089906F058FBBF
:108404003078FF282BD105E025EC0000CC0E0020AD
:10841400300D00200DA800780BA9497881421ED1A7
:108424000DA840780BA98978814218D10DA88078CD
:108434000BA9C978814212D10BA8457903480122BE
:10844400069905F009FEA84209D101E0CC0E0020EE
:108454000BA8007904990840602800D1EDE00DAD27
:10846400AF8010480D9010480222294605F0F4FD13
:10847400A8700BAEB7800B97204608993A4606F0D1
:1084840017FB0A9800900948062329463246FDF74F
:1084940095F801222046089906F00AFB3078FF2857
:1084A4002BD105E025EC0000CC0E0020300D00207F
:1084B4000DA800780BA9497881421ED10DA84078F7
:1084C4000BA98978814218D10DA880780BA9C978A5
:1084D400814212D10BA8457903480122069905F07F
:1084E400BBFDA84209D101E0CC0E00200BA8007905
:1084F40004990840602800D19FE00DADAF8010487A
:108504000D9010480222294605F0A6FDA8700BAE76
:10851400B7800B97204608993A4606F0C9FA0A989C
:1085240000900948062329463246FDF747F8012200
:108534002046089906F0BCFA3078FF282AD105E0D5
:1085440025EC0000CC0E0020300D00200DA8007892
:108554000BA9497881421DD10DA840780BA98978CF
:10856400814217D10DA880780BA9C978814211D115
:108574000BA8457903480122069905F06DFDA84230
:1085840008D101E0CC0E00200BA800790499084022
:10859400602852D00DADAF8010480D9010480222D3
:1085A400294605F059FDA8700BAEB7800B972046FD
:1085B40008993A4606F07CFA0A980090094806237E
:1085C40029463246FCF7FAFF0125204608992A4637
:1085D40006F06EFA3078FF2806D0C0E225EC0000E1
:1085E400CC0E0020300D00200DA800780BA949788E
:1085F400814200D0B3E20DA840780BA9897881426A
:1086040000D0ACE20DA880780BA9C978814200D0D3
:10861400A5E20BA8467904480122069905F01CFD41
:10862400B04203D09BE2C046CC0E00200BA80079D8
:1086340004990840602800D091E2089F10480D90EA
:1086440010480DAD0222294605F006FDA870099ACE
:108654000B922046394606F02BFA0A9800900A48F5
:108664000BAE0423294632460693FCF7A7FF0122EA
:108674002046394606F01CFA3078FF2819D105E067
:10868400F2EC0000CC0E0020300D00200DA8007884
:108694000BA9497881420CD10DA840780BA989789F
:1086A400814206D10DA880780BA9C978814200D1F6
:1086B400DBE010480D9010480DAD0222294605F06C
:1086C400CBFCA870099A0B922046394606F0F0F9C3
:1086D4000A98009009480BAE042329463246FCF759
:1086E4006DFF01222046394606F0E2F93078FF2872
:1086F40019D105E0F2EC0000CC0E0020300D002072
:108704000DA800780BA9497881420CD10DA84078B6
:108714000BA98978814206D10DA880780BA9C97864
:10872400814200D1A1E010480D9010480DAD022205
:10873400294605F091FCA870099A0B922046394607
:1087440006F0B6F90A98009009480BAE04232946AE
:108754003246FCF733FF01222046394606F0A8F9D9
:108764003078FF2818D105E0F2EC0000CC0E002090
:10877400300D00200DA800780BA9497881420BD157
:108784000DA840780BA98978814205D10DA880787D
:108794000BA9C978814268D0FB480D90FB480DAD08
:1087A4000222294605F058FCA870099A0B9220462B
:1087B400394606F07DF90A980090F5480BAE04237B
:1087C40029463246FCF7FAFE01222046394606F0D5
:1087D4006FF93078FF2811D10DA800780BA94978DA
:1087E40081420BD10DA840780BA98978814205D12B
:1087F4000DA880780BA9C978814236D0F7480D902E
:10880400F5480DAD0222294605F026FCA870099A08
:108814000B922046394606F04BF90A980090ED4831
:108824000BAE042329463246FCF7C8FE0125204638
:1088340039462A4606F03CF93078FF2800D0B2E1E8
:108844000DA800780BA94978814200D0ABE10DA8AE
:1088540040780BA98978814200D0A4E10DA88078E2
:108864000BA9C978814200D09DE10DAD099FAF806D
:10887400DB480D90D8480222294605F0EDFBA8708C
:108884000BAEB7800B97204608993A4606F010F9CC
:108894000A980090CF48062329463246FCF78EFEFC
:1088A4000125204608992A4606F002F9301D059054
:1088B4003078FF2824D10DA800780BA9497881428B
:1088C4001ED10DA840780BA98978814218D10DA832
:1088D40080780BA9C978814212D10BAE7779BE4852
:1088E40005992A4605F0B8FBC01B411E884106992C
:1088F4007156002900DA00252843012800D05EE1E2
:108904000DAD099FAF80B6480D90B34802222946A9
:1089140005F0A2FBA8700BAEB7800B972046089910
:108924003A4606F0C5F80A980090AA480623294654
:108934003246FCF743FE0125204608992A4606F0F4
:10894400B7F83078FF2824D10DA800780BA949780E
:1089540081421ED10DA840780BA98978814218D193
:108964000DA880780BA9C978814212D10BAE777912
:10897400994805992A4605F06FFBC01B411E8841A2
:1089840006997156002900DA00252843012800D0F1
:1089940015E10DAD099FAF8091480D908E480222DC
:1089A400294605F059FBA8700BAEB7800B972046FB
:1089B40008993A4606F07CF80A9800908548062300
:1089C40029463246FCF7FAFD0125204608992A4635
:1089D40006F06EF83078FF2824D10DA800780BA992
:1089E400497881421ED10DA840780BA9897881422B
:1089F40018D10DA880780BA9C978814212D10BAE89
:108A04007779754805992A4605F026FBC01B411E57
:108A1400884106997156002900DA00252843012867
:108A240000D0CCE00DAD099FAF806D480D906A4831
:108A34000222294605F010FBA8700BAEB7800B97F5
:108A4400204608993A4606F033F80A98009061489F
:108A5400062329463246FCF7B1FD01252046089934
:108A64002A4606F025F83078FF2824D10DA800788E
:108A74000BA9497881421ED10DA840780BA98978A9
:108A8400814218D10DA880780BA9C978814212D1EE
:108A94000BAE7779504805992A4605F0DDFAC01BDC
:108AA400411E884106997156002900DA00252843A1
:108AB400012800D083E00DAD099FAF8048480D9098
:108AC40045480222294605F0C7FAA8700BAEB780C4
:108AD4000B97204608993A4605F0EAFF0A98009059
:108AE4003C48062329463246FCF768FD012520460A
:108AF40008992A4605F0DCFF3078FF2823D10DA819
:108B040000780BA9497881421DD10DA840780BA9A2
:108B14008978814217D10DA880780BA9C978814240
:108B240011D10BAE77792C4805992A4605F094FAB1
:108B3400C01B411E8841069971560029294600DA56
:108B4400099908433BD0ED024B2086006436204649
:108B5400294605F0B5FF3046FAF784FBF7E7ED0246
:108B64004B2086002046294605F0AAFF3046FAF736
:108B740079FBF7E7F5022046294605F0A1FFC82056
:108B8400FAF770FBF7E7C046F2EC0000CC0E0020C9
:108B9400300D0020F5022046294605F091FFFA2009
:108BA400FAF760FBF7E7ED024B20860032362046E9
:108BB400294605F085FF3046FAF754FBF7E796207F
:108BC400FAF750FB01222046079905F071FF0FB018
:108BD400F0BDC046300D0020CC0E0020F2EC0000A9
:048BE40021EC000080
:108BE800F0B58BB008AE0025357209959F480890FE
:108BF8009F480222314605F02DFAB07005AF3D724C
:108C0800069505950520000703900124E1030491CA
:108C18000195002205F04AFF0A2000909548092393
:108C280031463A46FCF7C8FC03980499029401229D
:108C380005F03CFF3878FF2834D108A8007805A94A
:108C4800497881422ED108A8407805A989788142BF
:108C580028D108A8807805A9C978814222D105A819
:108C6800057A011D82480424224605F0F3F9A8423A
:108C780018D105A80057002814D5044012D0402167
:108C880001400FD1082108400CD105A841790904F9
:108C9800827912025218C0791318C80D0BD0774880
:108CA8001B1808E0C120400073490A5A521C0A5296
:108CB800FFF74CF8019B72480168724A914201D053
:108CC8004A1C0260019270480068C118C20F8018DF
:108CD80040100E1AF00F301847103120C000664BB4
:108CE8001F50986F03901C46C834E0680494802194
:108CF800595888229A58401A504303F0EBFE634BA8
:108D0800002203F047FD03F043FE632189005A4B1C
:108D180058505D490E600399791A5D4A1160091A25
:108D280003915C4801600420205E7E21595E1E4646
:108D3800401A03F0CFFE04460F469020305803F047
:108D4800C9FE22463B4605F0D4FC00224F4B03F0F7
:108D580021FD03F01DFE0399081A4F49086003F02E
:108D6800B9FE4E4B002205F0C4FC4D4B002205F025
:108D7800C0FC7D22D305002205F0BBFC06460F4649
:108D880048480660416094203B4C205803F0A2FEFE
:108D9800454B002203F0FEFC32463B4605F0A9FC99
:108DA80003900F46414981C106200499085E982125
:108DB800615E401A03F08EFE04460E46A4202E493A
:108DC800085803F087FE3A4B002203F0E3FC2246E2
:108DD800334605F08EFC374B002203F093FB039AD1
:108DE8003B4605F086FC06460F4633480660416060
:108DF800324B3046002203F08BFD00281BD10022A5
:108E08002F4B3046394603F0A3FD002813D100222A
:108E18001E4B3046394605F06CFC03F0B9FD029A4A
:108E2800019B049C144DE4216850152B0EDA25484B
:108E380002600BB0F0BD192000010F4D2858029AAE
:108E4800019B049CE4216850152BF0DBE069216A42
:108E5800884201DDE0692062E069616A8842E6DAF9
:108E6800E0696062174802600BB0F0BD12EC0000C8
:108E7800CC0E0020300D002030000020010000FF43
:108E8800BC0F0020FFFFFF7FC00F002000408F4075
:108E98006C0F0020740F0020700F002000000840A5
:108EA80000006940A005002080842E419005002024
:108EB80065CDCD410000F03F98050020003081408D
:088EC800003081C0400F0020C2
:108ED0000548C16D054A4A430521890142504018A1
:108EE000D11741607047C04630000020F0F1FFFF0D
:108EF000F0B589B0DD4DE86DE1210B01010C1C0CD2
:108F0000002208939BB2594380B2029343430394D7
:108F10000C0C0904591854410022002040180690F6
:108F200062410792D24B03CB083B014307D100209B
:108F30004B2189006958CF4A4A431A605860CE4B8A
:108F400003CB083B014307D10020132109016958D5
:108F5000C84A4A431A605860E424285900280594F6
:108F60000FD45220285A03F005FE0022C34B03F011
:108F700015FC06460F46285903F0B0FD32463B4625
:108F800030E0E86D6821695A03F07EFE06462959F3
:108F900028597242914229DA03F0A0FD04460F4697
:108FA0000491304603F09AFD02460B460120C107AA
:108FB0007940204603F0F2FB01900F465020285ADA
:108FC00003F0D8FD0022AD4B03F0E8FBAC4B0022D0
:108FD00003F09CFA02460B460198394603F038F933
:108FE0002246049B05F089FB03F0D6FC2C46C834CE
:108FF000A0627020285EA16A081AA062E169E06997
:10900000002913D4C1179C4D44CD083D17184E417B
:10901000984A00233846314603F072FE13210901B5
:10902000924A50502F606E60904D1BE0904A06CAE5
:109030004042C6170F1856418E4A00233846314623
:1090400003F05EFE4B218900685069587D20C00006
:109050004843E96D03F018FE4F21890068528448A7
:1090600007604660A06A616BC217236B1818206303
:109070004A416263A06AE16FC217A36F1818A06724
:109080004A41E267A06FE16F0026089A334603F079
:109090001FFE2D21C90004916850606B216B069A58
:1090A000511A0799814105DAF8202A502846F830EC
:1090B000079941600520800129184A682B585B1EDA
:1090C000B24102DB00222A504A60E96D5420285A3E
:1090D000D827EA595823EB5A9A4211DD484303F046
:1090E00049FD664B324603F059FB03F06FFC059ACD
:1090F000AA58D317101A8B4102DA62480088461C1E
:10910000604806805620285A31B281420BDD07980C
:109110006063069820630020E067A06702F044FDCA
:10912000594801210160206B616B0026089A334683
:1091300003F0CEFDE06220690321C901695A88422B
:1091400030DAE8597D21C90088422BDD4F4801887B
:10915000491C018089B20A2926D34B4C2168012978
:1091600022D10A2101800920400129580909E12959
:1091700013D32858464988420FD8049968580028C4
:10918000685800D5404243218900685002F02AFC0B
:1091900000212160284600F057FF4920800000216F
:1091A000295001E0394806806420285A042835D81F
:1091B00078440079400087440222282B2E00E86D75
:1091C0000023010C039C22464A43029E714380B255
:1091D000464360430F0C090471185741040C000406
:1091E00046187C41F82028582946F8314968294A10
:1091F00003F00AFD3246234603F06AFD0DE00499B0
:10920000685800280FD400200FE002F025FC04E08D
:1092100002F04CFC01E002F081FC06460120000255
:109220002E5009B0F0BD68584042432189006A5869
:10923000002A02DD6F58F91701E0EF6D0021089157
:10924000C117144E00243246234603F0DDFC3A4693
:10925000089B03F03DFD721E2346A341121A8B4169
:1092600000DB341A0029D9D42646D7E73000002085
:10927000B805002080EE3600C005002000005940EF
:109280000000F0BFC80F00203C0F0020C60F0020D8
:0892900080FC0A00A086010029
:10929800F0B583B00546354B1868354A904206D07C
:1092A800421C1A60334A904201DC002000E0012091
:1092B8000190314803681A0A9A1A541904602F4811
:1092C8000268130AD21A029152180260100A210A7F
:1092D800081A03F0FFFB06460F462E4C608803F081
:1092E80045FC32463B4605F004FA0022254B03F0C4
:1092F80051FA254A254B03F005F9254B002205F0C4
:10930800F8F903F045FB2061019800280BD020698B
:109318006169884201DD206960612069A16988422C
:1093280001DA2069A0610298281A03F0D3FB0446E9
:109338000D46CA20124E305A03F018FC22462B461E
:1093480005F0D7F900220F4B03F024FA0E4A0F4B11
:1093580003F0D8F80E4B002205F0CBF903F018FB08
:1093680065218900705003B0F0BDC046B00F0020E1
:10937800FFFFFF7FFF090000B40F0020B80F002097
:1093880030000020ECFF2341DA9E4A94EEBF90BFE4
:0893980000004540F800002030
:1093A000F0B581B0114F388803F0D4FB7321CC05A0
:1093B000214603F097F90E4E314603F093F903F07E
:1093C0003FFB05460B480560788C03F0C3FB214644
:1093D00003F088F9314603F085F903F031FB0649C3
:1093E0000860401B0549086001B0F0BDA875FF1F6B
:1093F00000803B45640F0020680F0020600F0020B4
:10940000F0B581B027494143080C27490968411A42
:10941000264848432649096803F00EFC25494018B0
:109420000A2103F009FCCC22234CA0525A21605A95
:109430000323DD016053A05E6A26A35F98422FDA02
:10944000A75AA25E6C20235E9A4200DC275A00973E
:10945000225E6E20235EA05F9042074606DD8242B8
:1094600007DA665E974208D1002018E0174682426C
:10947000F7DB0246665E9742F6D0B91AB342184649
:1094800000DB30460F4647439E4200DC1E46301A42
:10949000009B1BB29A1A4243D01903F0CDFB6053D4
:1094A00001B0F0BDE40C0000640F0020A0860100B4
:0C94B000600F002030750000300000202C
:1094BC0010B582B00848026801210A4302600068B6
:1094CC0008400190019809200022FAF789FC092034
:0C94DC00FAF7A2FC02B010BD38100240EC
:1094E80070B50121CB06104A12681206920BD518E6
:1094F8000E4BD418661C0324AE4213D8D25C002845
:1095080000D00270382A06D0FF2A07D0392A09D19C
:109518000948012404E00224064801E00024044824
:1095280003F07AFC204670BDE075FF1F00F8FF07C6
:0C95380034ED000848F300081DEF0008A7
:10954400F0B583B00190524803F068FC514E0125F8
:10955400358428044B210902B161F06130462A3078
:109564001E2104F005FCB8204B493150B4204B496E
:109574003150B0204A493150AC204A4A3250A820D8
:109584003150A4203250A020474931509C204749F3
:109594003150982046493150962002273752942062
:1095A4003554AF208001703092217052902041498F
:1095B4003152882040493150802040493150304652
:1095C40018303F4941673F49C1663F4900203F4A3F
:1095D400B264F06430657065B165BC217050D0210F
:1095E4007050CC215A2272523146BC314860886096
:1095F400C860C143364AFB43364C30667066B16678
:10960400F1663467304674300EC0D820706039205B
:109614003070B068401CB060FAF7F4FE7D20C000E2
:10962400FAF798FE2C480168C90702D00168A943DB
:1096340001602A4807602A4C21680906490E491E20
:109644008160C56002A9FAF785FF002800D0FEE713
:1096540020680006800B234C0519FF2087020CCEDE
:1096640001202946083EFAF79BFD0028FED11C483C
:109674000068800238402018D43008360835854206
:10968400EDD3FAF7D3FE019800F02EF803B0F0BD45
:109694004BEF0008E803002010270700320038FFD2
:1096A40054F248F44C1D581B0CFEF40160EAC0DA75
:1096B400C02BE02EB036000080482800630069000B
:1096C4000A000200A086010040420F0090D003006F
:1096D400007884C900D68AEA142002402C0F0020A6
:0896E400E075FF1F00F8FF070D
:1096EC00F0B59DB004460120C206D34909680906AD
:1096FC00890B8B18D14A8E183146D831994200D932
:10970C0095E10490432080002018029020464030C0
:10971C00009003948C340194701C1C90B01C1B9012
:10972C00F01C1A90301D1990701D1890B01D1790D8
:10973C00F01D1690304608301590304609301490C4
:10974C0030460A30139030460B30129030460C30B5
:10975C00119030460D30109030460E300F90304640
:10976C000F300E90304610300D90304611300C906A
:10977C00304612300B90304613300A90304614307D
:10978C000990304615300890304616300790304618
:10979C001730069030461830059033461933314651
:1097AC001A31D724E443A64805193219D827D25DBB
:1097BC00EA551C980219D25DD9202A541B9800191D
:1097CC00C05DDA22A8541A980019C05DDB22A85497
:1097DC0019980019C05DDC22A85418980019C05DB6
:1097EC00DD22A85417980019C05DDE22A8541698E3
:1097FC000019C05DDF22A85415980019C05DE02245
:10980C00A85414980019C05DE122A85413980019AB
:10981C00C05DE222A85412980019C05DE322A8543E
:10982C0011980019C05DE422A85410980019C05D6D
:10983C00E522A8540F980019C05DE622A8540E9892
:10984C000019C05DE722A8540D980019C05DE822EC
:10985C00A8540C980019C05DE922A8540B98001963
:10986C00C05DEA22A8540A980019C05DEB22A854E6
:10987C0009980019C05DEC22A85408980019C05D25
:10988C00ED22A85407980019C05DEE22A854069842
:10989C000019C05DEF22A85405980019C05DF02294
:1098AC00A8541819C05DF122A8540819C05DF22201
:1098BC00A8541B3400D076E7614DA8690399086160
:1098CC00A88B8882E88BC882288C0883688C888354
:1098DC00A88CC883E88C0884288D4884688D009CEB
:1098EC00A087A88DE087E88D019B9881288ED88170
:1098FC00688E1880A88E9882E88E9883A86B206456
:10990C00E86B6064286CA064686C5860A86C186183
:10991C00E86C9861286D1862686D8867A86D98600E
:10992C008020285A60828220285A208228461830AB
:10993C00C06EC8658820285808668C20285AA082DA
:10994C008E20285AE0829020285A20839220285A70
:10995C0060839420285CA0849620285A2085982027
:10996C00285A88869A20285AC8869C20285A088704
:10997C009E20285A4887A020285A8887A220285A37
:10998C00C887A420285A2080A620285A6080A820A6
:10999C00285AA080AA20285AE080AC20285A20817E
:1099AC00AE20285A6081B020285AA081B220285AB3
:1099BC00E081B420285A6085B620285AA085B820AA
:1099CC00285AE085BA20285A2086BC202858029AAA
:1099DC001062C02028585062C42028589062C820B9
:1099EC002858D062CC20285A6086D0202858D061C4
:1099FC00286ED866686E1867A86E1060E86E5060A6
:109A0C00686F9063286F5063E86F1064A86FD06321
:109A1C00E8684860A888D8280BD10948C088002875
:109A2C00049804D1064800783938411E88411DB08D
:109A3C00F0BD04981DB0F0BDE075FF1F00F8FF07E6
:049A4C00E80300200B
:109A5000F0B59FB00D460446EA4803F0E1F9012055
:109A6000C106E94A12681206920B5118E74BD21848
:109A70001346D0338B4201D91FB0F0BD0595019438
:109A8000FF2080020490901C1D90D01C1C90101D83
:109A90001B90501D1A90901D1990D01D18901046C3
:109AA0000830179010460930169010460A3015906D
:109AB00010460B30149010460C30139010460D30A9
:109AC000129010460E30119010460F301090104634
:109AD00010300F90104611300E90104612300D903D
:109AE000104613300C90104614300B901046153071
:109AF0000A9010461630099010461730089010460C
:109B00001830079016461936501C06900020039016
:109B1000C0430290CF38BE4909181518D023ED5C18
:109B2000CD54069C2518ED5CD1240D551D9C2418A0
:109B3000E45CD2254C551C9C2418E45CD3254C5580
:109B40001B9C2418E45CD4254C551A9C2418E45C16
:109B5000D5254C55199C2418E45CD6254C55189CE9
:109B60002418E45CD7254C55179C2418E45CD827AE
:109B7000CC55169C2418E45CD9254C55159C24180A
:109B8000E45CDA254C55149C2418E45CDB254C5528
:109B9000139C2418E45CDC254C55129C2418E45CCE
:109BA000DD254C55119C2418E45CDE254C55109C99
:109BB0002418E45CDF254C550F9C2418E45CE02558
:109BC0004C550E9C2418E45CE1254C550D9C241842
:109BD000E45CE2254C550C9C2418E45CE3254C55D0
:109BE0000B9C2418E45CE4254C550A9C2418E45C86
:109BF000E5254C55099C2418E45CE6254C55089C49
:109C00002418E45CE7254C55079C2418E45CE825FF
:109C10004C553418E45CE9254C551A3000D07AE7ED
:109C20001C97F749486DF74F7865488D7885888D82
:109C3000B885486B1B90886B1D900A463C3274CAED
:109C4000C86C1A90086D1990488E7886886DB86532
:109C5000C88DF885088E38861B9878631D9839461C
:109C6000383175C11A98F86419983865059D012D29
:109C700006D0E34EB0690399B861084607D107E002
:109C80004B2000020399DE4EB861084600E0B08B1D
:109C9000B883012D03D1FD8304D1632004E0F08B50
:109CA000F883FAD07820305A328C80217852012DF6
:109CB00009D0705888217850012D08D10A248C20B1
:109CC0003C5269240BE0D04888217850F6E7842084
:109CD000345A8C203C52012DF3D07A24345B8225F7
:109CE0007C53059D012D00D12A463A84012D039C09
:109CF00022460CD17A8422460DD1BA84012D224607
:109D00000ED1FA8422463A8513E0F26F12E0728C8B
:109D10007A842246F1D0B28CBA84012D2246F0D04A
:109D2000F28CFA84012D2246EDD0328D3A85012D38
:109D3000EBD1B64A3C461834E2660222012D1D9250
:109D400001D08622B25A8E243A53012D01D0715A85
:109D500000E0AF4990257953AF218901059A012A86
:109D600002D08A22B65A01E00E4670369222BE52C6
:109D7000059E012E1B9502D18E25344602E08E25CC
:109D80009F4C245C94203C54012E1D9C10D19625A0
:109D90007C539824395318E099498A5A9A217A5267
:109DA000012E16D19C4A9C203A529C4A944E18E0AF
:109DB000934C645B96257C53012EEAD090491B9C02
:109DC000095B98243953012EE6D1924A9A217A529E
:109DD000E8E78B4A125A9C203A52012EE5D0884E71
:109DE000725B9E257A53059A012A01D0325B00E00E
:109DF0008B4AA0243A537D24059A012A0AD0715A2D
:109E000009E0C04690F30008E075FF1F00F8FF0767
:109E1000C0040020A1001B94A2221992B9528149CA
:109E2000059E012E0A4601D0754A125AA4201890A8
:109E30003A527348445B7C4A012E00D02246A82047
:109E40001A903A52794A012E3046154600D02546DE
:109E5000A6243D53764D012803D0694D19996D5ABA
:109E60007049AA261996BD53012802D06449189D4D
:109E7000495BAC257953012801D061490A5BAE21C9
:109E80007A520128684C6A4E07D1B022BC52B224E3
:109E90003E5310E05A48455B0EE0594A1A9C145B49
:109EA000B022BC520128F2D0554C199EA65BB224B8
:109EB0003E530128EED132254F4EB4203D52059D30
:109EC000012D02D04E4D695A01E0C721C943B62584
:109ED0007953059D012D07D049498A5AB8217A52F4
:109EE000012D05D1072205E0524AB8217A52F9E73F
:109EF000434A125BBA243A53012D039C224601D0F7
:109F00003F4A1258BC203A50012D204601D03C480F
:109F10004058C0217850C420012D02D03849095A38
:109F200000E05A21CC22B952C821012D224601D08D
:109F3000334C6458FC507A503A501D98C0433E4907
:109F40003E4B3A667A66029CBC66FC663B677C6761
:109F5000B967F8672A498868401C88601C9979604D
:109F6000B86039203870012D01D02548027C3A7440
:109F7000012D1B9C02D02248C06803900398F86012
:109F8000FAF742FAE000FAF7E7F92D480168C90745
:109F900003D001680122914301602A480221016037
:109FA000316801220906490E491E8160C2601EA95E
:109FB000FAF7D2FA0028114C00D0FEE73068800290
:109FC0000499084005190CCF01202946083FFAF7EB
:109FD000E9F80028FED13068800204990840201872
:109FE000D430083708358542EDD3FAF721FA0198C5
:109FF000FFF77CFB1FB0F0BDE075FF1F00F8FF0707
:10A00000C0040020E803002080482800A08601004A
:10A01000B0360000E02E000060EAFFFFC0DAFFFF6C
:10A020000CFEFFFF4C1D000054F2FFFF581B000008
:10A0300048F4FFFF10270000007884C900D68AEAA0
:08A04000142002402C0F002047
:10A04800F0B583B001910446804802F0E5FE20692E
:10A058007F4EB061A08AB083E08AF083208B308481
:10A06800A08B7084E08BB084208CF084608C308569
:10A0780021464031C88FB085888F708520468C3046
:10A088008289F285C28932868C22A35A7386838A92
:10A09800B386838BF3860B6CB3634B6CF3638B6C67
:10A0A8003364436873640369B3648369F364036A5C
:10A0B8003365A36F73658368B3654B8A8027F35351
:10A0C8000B8A8227F353E36D37461837FB66236EF6
:10A0D8008827F3518B8AB352CA8A8E23F2520A8B8D
:10A0E8009023F2524A8B9223F2528A8C9423F25490
:10A0F8000A8D9623F252A28E9823F252E28E9A2368
:10A10800F252228F9C23F252628F9E23F252A28F28
:10A11800A023F252E28FA223F2524022A25AA42391
:10A12800F2524A88A623F2528A88A823F252CA8891
:10A13800AA23F2520A89AC23F2524A89AE23F25278
:10A148008A89B023F252CA89B223F2524A8DB423C3
:10A15800F2528A8DB623F252CA8DB823F2520A8E71
:10A16800BA23F25243229300E218176ABC257751AA
:10A17800556AC027F551956AC427F551D56AC8278D
:10A18800F551498ECC257153D169D0257151016F94
:10A198007166C06E3066E058B0665068F066506B05
:10A1A8003067906B7067D06BB067106CF0673920C0
:10A1B8003070D8207060B068401CB06001980028EA
:10A1C80004D0244802F028FE6068F060FAF718F915
:10A1D8007D20C000FAF7BCF81F480168C90703D002
:10A1E80001680122914301601C48022101601C4D55
:10A1F800296801220906490E491E8160C26002A928
:10A20800FAF7A6F9002800D0FEE728680006800BB8
:10A2180014494518FF2087020CCE01202946083E24
:10A22800F9F7BCFF0028FED10D48006880023840CD
:10A238000C490818D430083608358542ECD3FAF7AB
:10A24800F3F82046FFF74EFA03B0F0BD61EF0008BF
:10A25800E803002045F10008142002402C0F0020DC
:08A26800E075FF1F00F8FF077D
:10A2700070B54F2080000F4E305A002816D0C836D7
:10A28000F06E02F077FC04460D46306F02F072FC6F
:10A2900002460B462046294602F080FA0022074B70
:10A2A00004F02BFA02F078FB00B270BD024800B255
:10A2B00070BDC04630000020FFFF00000000594084
:10A2C000F0B58BB088480068884A1446C834216EBF
:10A2D000081ACD2149005052854D281D7C2229465F
:10A2E00003F052FD834F381D39467C2203F04CFDAC
:10A2F000E069099028602069386000207E4B0446A0
:10A300000246194606E0001D802833460A9C3A465C
:10A31000294619D0774D2D58EE177540AE1BA64231
:10A32000354600DC25460A959E42714C00DB1E46F0
:10A330002358DC1763401D1B95422F4600DC17464F
:10A340008D42E0DB0D46DEE7781BC1174840441A1A
:10A35000664AD06D6821515A02F096FC142102F031
:10A360006BFC844205DA0120C043401C00B20BB0F4
:10A37000F0BD0A98801BC1174840401A192803D223
:10A380005E4800B20BB0F0BD08900A945D4900220F
:10A39000D7433D4601E0521C10310B1F1E6809983F
:10A3A000331ADC1763401C1BAC42104600DC3846F5
:10A3B0000F68BE1BF3175E40F61AAC421DDDA642C5
:10A3C0001ED8A64200DC26464D68EB1BDC17634016
:10A3D0001C1BB44200D9901CD21C1F2A1DD08B68B4
:10A3E00009935B1BDD176B405D1BB4420CDDA5427E
:10A3F00017460DD9A542CEDC0DE02C46A642E0D989
:10A40000501CA642DFDDDFE73446A5421746F1D8EF
:10A410000746A542BFDC2546BDE7102860D1089855
:10A4200002F05CFB04460D460A9802F057FB024618
:10A430000B462046294602F0B1F90024304B224653
:10A4400004F05BF902F0A8FA47218900274A50522C
:10A450002520C0001058244908604320C00010186F
:10A4600001940021224C6258C261224D6B58024671
:10A470008032D36163185C689E680596DE68069634
:10A480001E6907965E6908969E690996DB690A93BC
:10A4900084616C18231DE8CB029767690397A7694D
:10A4A0000497E4699361059B43615561069B0361D1
:10A4B0001661079BC360029BD360089B8360039B6C
:10A4C0009360099B436057600A9A0260802284501F
:10A4D000203820318029C5D1019800B20BB0F0BDE1
:10A4E00000200BB0F0BDC046A40F002030000020BB
:10A4F000B00C0020B00B0020FFFFFF7FFEFF00002C
:08A5000000408F40B80C002060
:10A50800F0B58BB08A4800688A4A1446C834216E70
:10A51800081ACD2149005052874D281D7C22294612
:10A5280003F02EFC854F381D39467C2203F028FCA9
:10A53800192000017F49085809902860E0683860B0
:10A5480000207F4B04460246194606E0001D80287D
:10A5580033460A9C3A46294619D0784D2D58EE17AD
:10A568007540AE1BA642354600DC25460A959E423C
:10A57800714C00DB1E462358DC1763401D1B9542B7
:10A588002F4600DC17468D42E0DB0D46DEE7781BE0
:10A59800C1174840441A674AD06D6821515A02F0E1
:10A5A8006FFBC117890F40188010844205DA01201B
:10A5B800C043401C00B20BB0F0BD0A98801BC11705
:10A5C8004840401A642803D25E4800B20BB0F0BD80
:10A5D80008900A945D490022D7433D4601E0521C89
:10A5E80010310B1F1E680998331ADC1763401C1BB7
:10A5F800AC42104600DC38460F68BE1BF3175E40BD
:10A60800F61AAC421DDDA6421ED8A64200DC26463C
:10A618004D68EB1BDC1763401C1BB44200D9901C2F
:10A62800D21C1F2A1DD08B6809935B1BDD176B405A
:10A638005D1BB4420CDDA54217460DD9A542CEDC00
:10A648000DE02C46A642E0D9501CA642DFDDDFE72C
:10A658003446A5421746F1D80746A542BFDC254631
:10A66800BDE7102860D1089802F034FA04460D4678
:10A678000A9802F02FFA02460B462046294602F0B5
:10A6880089F80024304B224604F033F802F080F9B0
:10A698008F214900274A50522520C00010582449CC
:10A6A80008606320C000101801940021224C6258F1
:10A6B800C261224D6B5802468032D36163185C68D0
:10A6C8009E680596DE6806961E6907965E69089676
:10A6D8009E690996DB690A9384616C18231DE8CB8F
:10A6E800029767690397A7690497E4699361059BD3
:10A6F80043615561069B03611661079BC360029B1A
:10A70800D360089B8360039B9360099B43605760F9
:10A718000A9A026080228450203820318029C5D1CD
:10A72800019800B20BB0F0BD00200BB0F0BDC046E0
:10A73800A00F002030000020300C0020300B00203B
:10A74800FFFFFF7FFEFF000000408F40380C002015
:10A7580070B5134A1368134CA34201D05B1C1360F5
:10A76800401A02F0B7F904460D46CA200E4E305A78
:10A7780002F0FCF922462B4603F0BBFF00220B4BEC
:10A7880002F008F80A4B002202F004F8094A0A4BC2
:10A7980002F000F802F0FCF819210901705070BDB0
:10A7A8009C0F0020FFFFFF7F30000020ECFF2341BB
:0CA7B80000004440FCA9F1D24D62203F9B
:10A7C400F0B58BB000240A94099438480168022239
:10A7D4001143016001681140059105990168042243
:10A7E4001143016001681140059105990168202217
:10A7F40004921143016001681140059105990168B3
:10A804000126314301600068304005900598052019
:10A8140000070190F9214D012946224604F048F928
:10A82400234F102103913846224604F041F93102A6
:10A8340002913846224604F03BF908962120000490
:10A8440007907002069006AF19483946F9F780FF61
:10A85400099408940796069501983946F9F778FF04
:10A86400089607944020069012483946F9F770FF7D
:10A87400099408940796029806900D4D2846394687
:10A88400F9F766FF099408960796039806902846F8
:10A894003946F9F75DFF09940896079604980690DF
:10A8A40028463946F9F754FF0BB0F0BD3410024086
:08A8B4000004005000080050F0
:10A8BC0001214A02904201D1014801607047C04613
:04A8CC00400F002019
:10A8D000A6B000261F961E961D961C961B961A96CD
:10A8E000199619A8F9F70EFF1D98AA2805D0CC28AB
:10A8F00005D0BB2806D1D54802E0D54800E0D548B0
:10A9000002F08EFAF8F764FC1F961E961D961C96B0
:10A910001B961A961296119610960127B80205906A
:10A92000FAF710F8F9F7FAFFCB4A506A18210143F9
:10A930005162F9F7FDFF78072590780424900820EC
:10A940002390229602242194209440201E901D964C
:10A950003D021C951B9706200290199019A8FAF742
:10A9600035F818961796169407200390159015A899
:10A970000221FAF73BFA04951495B80713900F9645
:10A98000B6480E900EA8FAF789FBB54802F048FACF
:10A99000FCF7C8F8FCF7D0F8FBF786FFFFF712FFCB
:10A9A000FEF78CFD00F0BAFDFCF7CEFE00F08CFC4B
:10A9B0003903A94C206808432060AA480A97076217
:10A9C000FF221023039D8560C3600261466186619A
:10A9D00002328280A44A026022680A4019921999C0
:10A9E000F9F756FA00F048FE00F014FFFEF770FA8F
:10A9F0000EAC2046FEF778FD9C4948802278CA813B
:10AA0000032811D8784400794000874401050901E2
:10AA10009648FEF797FD07E09448FEF767FE03E0CF
:10AA2000F3480021FFF714F8F24802F0F9F9F04C6E
:10AA30002046FEF75BFEF04D4021284603F06FFCF8
:10AA400000280FD13220F8F70FFC4021284603F0F0
:10AA500066FC002806D1E94802F0E2F9E448012149
:10AA6000FEF7F6FF2169A28AE38AE5480090E548EF
:10AA700004F030F8FEF794FC2546E34C2046F8F746
:10AA80006BFFE24908222046F8F7C4FDE04804992C
:10AA90003A4604F00FF86420F8F7E6FBFDF75AF9A0
:10AAA000DC4802F0BDF900F087FA052001900407A8
:10AAB000288B00281CD0F8020C9007460D96012226
:10AAC0002046394603F0F6FF2E46049D5E352846A3
:10AAD000F8F7CAFB00222046394603F0EBFF284670
:10AAE00035460D9EF8F7C0FB761C288B8642E5D3D1
:10AAF000079400262846C83006900C960B962C46E4
:10AB0000374603E084202221BD4A1150C248006824
:10AB1000012823D10025C04805603C46BB4F786919
:10AB200000F0B0FB386800F0DFFC7868B968FEF729
:10AB3000B3FBF8683969FFF70FFE069F3A69D31730
:10AB4000F869C11702F060F87D22D200002302F0FC
:10AB5000BFF838642746A64CFFF7D6FCAF4800681C
:10AB6000012806D103F0DAFFFFF7AAFB0020AB496A
:10AB70000860F8F773FB0146A9480068056840685B
:10AB80000D918E1B701E8641002F0A9A00DC002258
:10AB90000F2005400C98854239D00892099725204E
:10ABA000C700E059401CE0510B98002803D10798DA
:10ABB000059903F087FFFEF79BF900F03BFE00F0DC
:10ABC00003FA00F0AFFAE059964902F05DF89649B1
:10ABD0000968884205D09449086000212046FFF7A3
:10ABE00033FA67202746840000F0C8FB38538B20D7
:10ABF0004400FFF73DFB38533C46844FF869FEF7AD
:10AC0000FFFBB86900F046FC0C95099F089A2620C6
:10AC10007C49085C618B002900D1A9E0002800D0A4
:10AC2000A6E0608B8149884222DC1546401E0A2836
:10AC300000D98BE078440079400087440533373CE5
:10AC400087D04044484B4F00002127E004F400081F
:10AC5000E8F3000820F40008381002400140020028
:10AC60004BED0008CC0E00200030024030000020E8
:10AC70006F491546884209DC6F49884231D06C49DA
:10AC8000884263D1012000F0EDF86EE0FD218900DB
:10AC900088422AD06749884258D101212046FFF7CF
:10ACA000D3F962E02046FEF74DFC5EE0012120462C
:10ACB000FEF7CEFE59E02046FEF718FD55E020468F
:10ACC000FCF7E4FE51E02046FCF7F8FE4DE0FCF70F
:10ACD0000FFF4AE02046FCF727FF46E0FCF7A6FFFF
:10ACE00043E0002000F0BEF83FE000201F901E90DF
:10ACF0001D901C901B901A90199019A8F9F702FD4D
:10AD0000019800061F90039800061E90BB201D901E
:10AD100002981990F9F778FB002802D0474802F012
:10AD20007FF8F9F7C5FB002802D0454802F078F813
:10AD3000444802F075F819A8F9F76EFC002807D00E
:10AD4000414802F06DF8F9F7C7FB0EE044480AE00D
:10AD5000F9F7C2FB3D4802F063F8F9F769FB3C489C
:10AD600002F05EF83B4802F05BF82A460020608360
:10AD70003240BF1A4021204803F0D1FA002819D1EF
:10AD8000002F079D16D10A20F8F76EFA40211A48C5
:10AD900003F0C5FA00280DD1049FF4370B98002862
:10ADA00002D000200B9005E00122284605990B9265
:10ADB00003F080FE134803F0AFFE00280D9E00D183
:10ADC000A4E61048FCF7A6F9022800D09AE60B98F2
:10ADD000002800D09AE60B48FCF78AFA96E6BFF303
:10ADE0004F8F1D481D490160BFF34F8F00BFFDE726
:10ADF00030000020B0F3000800080050C0F3000845
:10AE0000A40A0020C8050020940D0020F00E0020A8
:10AE10000004005077EF0008440F0020400F00208E
:10AE2000A00E0020805101007C0F0020F1030000E3
:10AE3000F3030000D2040000F2030000D4F3000882
:10AE40005AED000884F1000885EF000895F100082C
:10AE500071ED0008AEF100080CED00E00400FA0509
:04AE600052F10008A3
:10AE640030B587B0054600240694059404940394F1
:10AE74000294019400946846F9F742FC002D27D00F
:10AE8400444801F0CBFF0498AA2832D1BB20049097
:10AE940002200090F9F7B6FA002802D0344801F0F5
:10AEA400BDFFF9F703FB002802D0334801F0B6FFD9
:10AEB4003A4801F0B3FF6846F9F7ACFB00281AD012
:10AEC400374801F0ABFFF9F705FB002007B030BDB0
:10AED4000498BB281CD1AA20049002200090F9F702
:10AEE40091FA002817D0224801F098FF002007B0FB
:10AEF40030BD29480AE0F9F7EDFA234801F08EFF46
:10AF0400F9F794FA214801F089FF264801F086FFF9
:10AF1400012007B030BD174801F080FFF9F7C6FAE9
:10AF2400002805D0144801F079FF002007B030BD97
:10AF3400124801F073FF6846F9F76CFB002807D04C
:10AF4400F9F7C8FA0E4801F069FF002007B030BDD8
:10AF54000C4801F063FFF9F7BDFA0B4801F05EFFFE
:10AF6400F9F764FA094801F059FF0948CEE7C046E9
:10AF7400D4F3000880ED00085AED0008B9EF00088A
:10AF8400CFEF0008CFF1000895F1000871ED00083B
:10AF9400F1EF000863F100089BEF000884F100085A
:08AFA40085EF0008AEF1000882
:0CAFAC000148012101607047440F0020A3
:10AFB80002480021C943C18781877047F8000020F3
:10AFC800F0B583B074244C4D285B002804D0285B6E
:10AFD80001281AD101221AE0484800880028484868
:10AFE80002D083214900685283214E00A95B0029C1
:10AFF80002D0A95B814250D1D8202858A98E0127B8
:10B0080088420FDA3F4802973DE0285B002205207E
:10B0180000070121490203F049FD285B37490880F0
:10B0280003B0F0BDE42028583C21695E7D22D2009F
:10B038004A43904203DA02200290334823E0CE21AB
:10B048006A5E48202B5E9A4203DD032002902F4857
:10B0580019E00197CC22AB5E285E83422C4802DDC2
:10B06800042102910FE06B5E4C216F5EBB4203DA54
:10B0780005200290274805E0AA5E695E8A420CDA3C
:10B0880006210291019F01F0C7FE0298A8530520EE
:10B0980000077902002203F009FDA85B0028BCD054
:10B0A800D8202858E98E8842B7DDE42028583C216A
:10B0B800695E7D22D2004A439042AEDDCE20295EF1
:10B0C8004A22AB5E9942A8DACC216B5EAA5E934213
:10B0D800A3DA2A5E4E202B5E9A429EDD695E285EC8
:10B0E80081429ADDA85B022897D00B4801F094FEB4
:10B0F8000020A85301228AE730000020C40F002056
:10B10800FFFF000013F00008ECF1000893ED0008C1
:0CB1180035F000083CF40008B6ED00081B
:10B12400F0B581B076244C4D285B002804D0285B10
:10B1340001281AD101221AE048480088002848480A
:10B1440002D041218900685241218E00A95B002967
:10B1540002D0A95B81424FD1D8202858298F0127DA
:10B1640088420FDD3F4800973CE0285B0022052021
:10B1740000070121090203F09BFC285B3749088082
:10B1840001B0F0BDE42028583E21695E7D22D20042
:10B194004A43904203DD02200090334822E0CE204F
:10B1A400295E4022AB5E994203DD032000902F48C4
:10B1B40018E0CC216B5EAA5E934203DD042000906C
:10B1C4002B480FE02A5E44202B5E9A4203DA0520C6
:10B1D4000090284806E0695E285E81420CDA062069
:10B1E4000090254801F01AFE0098A8530520000796
:10B1F4003902002203F05CFCA85B0028BDD0D820F3
:10B204002858698F8842B8DAE42028583E21695EBC
:10B214007D22D2004A439042AFDACE20295E4222F8
:10B22400AB5E9942A9DACC216B5EAA5E9342A4DAA2
:10B234002A5E46202B5E9A429FDD695E285E81422B
:10B244009BDDA85B022898D00C4801F0E7FD0020A4
:10B25400A85301228BE7C046300000202A000020BA
:10B26400FFFF000005F2000826F20008C5ED000803
:10B2740057F0000860F4000879F00008E8ED0008D1
:10B28400F0B581B00A4D29688A09891A0E18B409E3
:10B2940008486043084901F0F5FC094F38802E60E6
:10B2A4000648214601F0EEFC788001B0F0BDC046AE
:10B2B400900F0020E8800000FFFF0000D08A2F7567
:04B2C400F80000206E
:10B2C80010B586B01A480024FF217F22194B03606D
:10B2D80001239B078460C260016144618461C46189
:10B2E800036244620394029401940094F9F78EFF78
:10B2F800002801D003F0DBF901A98C700220088036
:10B308000594049402940A480122FAF72FF80028B9
:10B3180001D003F0CCF9084800900548694601229D
:10B3280002F0FFFF002801D003F0C1F906B010BDFC
:0CB33800A00E00200028004001041618A0
:10B3440081B000680A49884201D001B070470120E9
:10B354008102084A13680B43136013680B4000937F
:10B364000099C003116A0143116201B07047C046DD
:08B37400002800403C100240DB
:10B37C00F0B581B05821384E705A745ACF2149001B
:10B38C00364D2F68775201F0EFFB354A354B03F001
:10B39C00AEF901F0FBFAD8217658864202DD002086
:10B3AC0028600DE0204601F0DFFB2F4A2F4B03F005
:10B3BC009EF901F0EBFA86420ADA00202749086070
:10B3CC002B4908600120C043411C08B201B0F0BDFC
:10B3DC0027480168002906D00A460A32964208DD41
:10B3EC0000211E4A0AE0066031460A460A3296429D
:10B3FC00F6DC0A398E42194A06DA00211160016026
:10B40C00204908B201B0F0BD781C1060194988427F
:10B41C00114D04D3E42028582321C900685225205B
:10B42C00C0002858144901F029FC144A1368002163
:10B43C009842CAD02323DB00EB5E114C2668B70977
:10B44C00F61BF3189E098D277F00EE5310602360C6
:10B45C00002001B0F0BDC04630000020880F002055
:10B46C007B14AE47E17AF03F0AD7A3703D0AEF3F59
:10B47C00800F0020312A000080510100840F002031
:08B48C008C0F0020FEFF000000
:10B4940010B511494143C817000C08180014642161
:10B4A40041430E4808180A2101F0C4FB0C4A114616
:10B4B400C831C88006200B5E08240C5F085EA342D6
:10B4C40002DDD021505210BDD223D25E904201DA67
:10B4D400C888488110BDC046E40C0000A015FFFFD9
:04B4E4003000002014
:10B4E800B0B5C1170A4D6A88002301F089FB1522FF
:10B4F800002301F085FB01F047FB044B002201F01B
:10B5080049F901F0ABFAE860B0BDC046000024413B
:04B51800F800002017
:10B51C0070B50F4800210162416281620722C2624C
:10B52C0001634163102301240A4D0560A504120236
:10B53C004126B60046608160C2600246103232C2BB
:10B54C00C361F9F7BBFF002801D003F0AEF870BD62
:08B55C00300D00200030014019
:10B5640070B58AB000681A49884201D00AB070BD2B
:10B57400012420031749CA680243CA60CA6802400A
:10B5840005920598086820430860086820400090E8
:10B59400002609960896079602200690E02005905A
:10B5A40000980520050705A92846F9F7D1F804965F
:10B5B400039602960194E003009069462846F9F741
:10B5C400C7F820212846012203F072FA0AB070BDA0
:08B5D400003001403410024078
:10B5DC0082B0094841680122114341604168114021
:10B5EC0001910199110702680A4302600068084042
:0CB5FC000090009802B070473C10024024
:10B6080010B5F7F71BFE0B4C2068401C2060C008E3
:10B618007D280DD3F7F71EFE0749884208D307484F
:10B62800C16D491CC16500212160816D491C81657E
:10B6380010BDC046780F0020214E0000F800002001
:10B6480080B50248F8F738FD80BDC046F80D0020E7
:10B6580080B50248FBF720FC80BDC046A40A002044
:10B6680080B50248FAF70CFC80BDC046540E002095
:10B6780010B5FF204100174801800246C83200215A
:10B68800D165916545239B00CC43C45254649464AE
:10B6980047239B00C4528F235B00C4522323DB0043
:10B6A800C4528D235B00C4520223038101234381CA
:10B6B80005238381084B5C1C14625362074B5C1C96
:10B6C80014815381064C54619361C1225200815206
:10B6D80010BDC04630000020FFFFFF7FFF7F000045
:04B6E8000080FFFFE0
:10B6EC00B0B51E4D2C1F20688006400F411E03294B
:10B6FC0022D81B487944097949008F442301171A31
:10B70C00296803220A40032A00D0164829684906F2
:10B71C00490F491C01F0B2FA29684904490E484303
:10B72C002968490F491C01F0A9FA0BE07D200002A1
:10B73C0008E00120C00305E00C3D28688004410F9F
:10B74C000848C84008490860226892093C23134005
:10B75C00064AD258D0400860B0BDC0460C1002401A
:10B76C0000127A000024F4002400002054DE0008AB
:10B77C00F0B587B000682149884201D007B0F0BD10
:10B78C000127B8031E49CA680243CA60CA6802404E
:10B79C00029202980868022528430860086828402D
:10B7AC00019004200690002405940494039508202D
:10B7BC0002900198134802AE3146F8F7C5FF069483
:10B7CC00059404970395402002900E483146F8F7F3
:10B7DC00BBFF0694059404940395802002900948BD
:10B7EC003146F8F7B1FF1B2000210022F8F7F8FAD8
:10B7FC001B20F8F711FB07B0F0BDC0460038014024
:08B80C0034100240000400505A
:10B814000548016E054A4A432921C900425040188F
:10B82400D11741607047C04630000020F0F1FFFF9F
:10B83400F0B589B0664A0ACA0846083A184307D1DF
:10B8440000234D20800063490858634941430AC2DC
:10B854000191624A12CA0846083A204307D10024DB
:10B864002720C0005B4908585B49414312C2039139
:10B874000494E420574C2158002902930ED47221D9
:10B88400615A20584843642101F0D4F95F218900AA
:10B8940060507020205E6158081A01E0F0202058A2
:10B8A4005F21890060506258D317D8202058C117EF
:10B8B40001F0A8F97D22D20000230092079301F041
:10B8C40005FA17221501059566190896276E726800
:10B8D4006359C31863514A4172602922D200A318E4
:10B8E4005C683C4DAE583018A8504C415C60E12077
:10B8F4000401380C00260694A4B26043BFB27C4312
:10B90400050C000421187541324E002000246118F2
:10B914006841089C6468059FF5594D1B0546A5417F
:10B924003C4602DA3151089948605868B158491EBA
:10B934000799884101DBB1505960B0585968002318
:10B94400069D2A4601F0C2F95B21890070503059E6
:10B95400089949682A46002301F0B8F92F21C90043
:10B9640070502120C00031583058002912D4C1171A
:10B97400039A1418049D4D41174A00232046294672
:10B9840001F0BCF92721C9007050144804604560D7
:10B9940009B0F0BD4042C117019A1418029D4D41EF
:10B9A4000D4A00232046294601F0A8F93146C83142
:10B9B400C866496E00984843F16D01F063F94F2160
:10B9C4008900705202480460456009B0F0BDC04669
:10B9D400A80500203000002080EE3600B0050020CD
:10B9E400F0B581B05B208000184C21582058002904
:10B9F40000D540422146C8318864496C1448002966
:10BA04001ED44321890061587D22E36D994216D2E8
:10BA1400E36D002B14D0D00000230A0C002680B262
:10BA240042438FB27843150C11044018754100212C
:10BA3400002210186941E26D01F060F900E0D000C5
:10BA440045218900605201B0F0BDC046300000209D
:04BA5400FFFF0000F0
:10BA5800F0B581B01149086E00281CD0E12212010E
:10BA68000023040C002692B2544380B24243270CB0
:10BA78002404121977410024002085187C411720DE
:10BA88000201885889184968054A01F0B9F82A4618
:10BA9800234601F019F901B0F0BDC046300000207E
:04BAA800A086010073
:10BAAC00F0B581B05B20800016490A58002A01D4F9
:10BABC00002001E008584042112212018B58002B43
:10BACC0002DD8D58EE1701E00D6E0026C1170E4FEA
:10BADC007A1C0024234601F091F82A46334601F0E3
:10BAEC00F1F802460948BB1A23468B4103DA0029B8
:10BAFC0004D501B0F0BD841A0029FAD4204601B057
:10BB0C00F0BDC046300000209F860100A0860100D9
:10BB1C00F0B581B0112003011E4AD058002808DD71
:10BB2C004320800010582D21C90051580818C11706
:10BB3C0005E0D06D2D21C90051580818002114467C
:10BB4C00C83426690325ED01575BA46C012C02DB7C
:10BB5C00D458E51701E0146E0025F219D30FD31851
:10BB6C005A10DB1701F04AF87D22D200002301F0B5
:10BB7C00A9F8094E3246002301F040F822462B4624
:10BB8C0001F0A0F8C1178843B04200DB304601B089
:0CBB9C00F0BDC04630000020A086010073
:10BBA80070B51248026EE1210B010021140C002629
:10BBB8009BB25C4392B25343250C24041B19754174
:10BBC80000240022D2186C4117231B01C250C2184E
:10BBD80054602922D2008150821851605B22920061
:10BBE800815009225201815070BDC04630000020AA
:10BBF800C20F490089184000034A40428A4101D3D4
:0CBC080000207047012070470000E0FFA2
:10BC14000122D2079143034A4A401043414248411A
:08BC24007047C0460000F07FEC
:10BC2C00074A0A40531E9A41C00F4900081805499B
:10BC3C00884201D3002000E0012010407047C0462C
:08BC4C000000F07F0000E0FFA2
:10BC540030B50E4B5D1C0C0D2C4010D0AC420ED0F8
:10BC6400A2189A4205DD0120C007014009480918BD
:10BC740009E0002A04DD064B19401205114330BDCA
:10BC84000120C0070140002030BDC046FE0700006F
:08BC9400FFFF0F800000F07FAC
:10BC9C0010B54B005B0D084CA34201D0002B02D118
:10BCAC000023136010BD054C1B191360044A11408E
:10BCBC00044A891810BDC046FF07000002FCFFFFB4
:08BCCC00FFFF0F800000E03FC4
:10BCD400F0B587B00E4604460021C843574F06907E
:10BCE400401C0590384601914841590004914D0D7E
:10BCF400534900D18CE0E50F710002914919039179
:10BD0400650006994D1B03998F4100D282E0D10F43
:10BD1400049D69185500059F7D1B88417AD3012134
:10BD2400C807304004904748354605400340101B7F
:10BD34001846A84171D2039109050298470D05914F
:10BD440003D0481E06400E430DE08D420AD20398EC
:10BD5400C004E10F6E00761864007F1E85423546EC
:10BD6400F7D300E02E461D0D3748054004D0059951
:10BD7400481E03400B430FE0059883420CD20398FE
:10BD8400C00406901946D30F4800C31852006D1E14
:10BD9400069881421946F6D3AF4212DDA01A314605
:10BDA400994104D454405E40264302D113E0204616
:10BDB4003146C40F49000E1944007F1EAF42EDDC2A
:10BDC4002F462046841A35469D41059906D4504095
:10BDD4005E40064304D1019C049916E004463546AE
:10BDE4000D420AD10398C004E10F6A00511864009F
:10BDF4007F1E05420D46F7D000E02946002F15DDD1
:10BE0400781E049A891800050918204607B0F0BD69
:10BE1400019CFAE7019C0A49F7E762405D4015433B
:10BE240000D00496002DD7D10024D5E70398C21B77
:10BE3400204600F0C7FE04460020E2E7FFFFDFFFD4
:0CBE44000000F87FFFFFFF7FFF070000F9
:10BE5000F0B583B00D46044628494A1C280D104011
:10BE6000421E8A4240D22749884205D20024002D32
:10BE7000264635DA264E33E03331884201D92E4644
:10BE80002EE01F49461820462946324600F08CFE17
:10BE90001D4A114001434A424A410020002D01DA67
:10BEA000014600E0012111430291184901903246F8
:10BEB00000F09AFE074632460E462E402740019B70
:10BEC000D843401C1049594100F07EFE029A3818B0
:10BED0007141002A00D10E46002A00D107463C4697
:10BEE0002046314603B0F0BD002802D10121C90728
:10BEF0000D402E460028F3D10024F1E7FE07000094
:10BF000001FCFFFFFF030000FFFF0F000000F0FF38
:04BF10000000F0BF7E
:10BF1400F0B587B00A0D521E484B9A4214D206AAB5
:10BF2400FFF7BAFE06460F464948301A4748814192
:10BF3400069C3046394618DA0022474B00F0E4FAF2
:10BF440006460F46641E14E0C30F4A00D31844008B
:10BF540064423B4C9C416AD3520D6CD000290A4682
:10BF640000DA394A002963DA66E00022394B00F02E
:10BF7400CBFA059403900D460024E2430494304622
:10BF84003946FFF765FE354B002200F0BDFA024644
:10BF94000B460398294600F0FFFB03900F46024628
:10BFA4000B4602F0A8FB04460D462D4E02213046F6
:10BFB40022462B4602F0D6FD2A4A2B4B00F0A4FA67
:10BFC4000290019110360321304622462B4602F09E
:10BFD400F1FD02460B460298019900F0DDFB224672
:10BFE4002B4602F088FB039C22463B4602F083FB6F
:10BFF40022463B4600F088FA06460F46059800F0B4
:10C004006BFD04460D46194A194B02F074FB324687
:10C014003B4600F079FA06460F46164B2046294661
:10C02400049A02F068FB32463B4600F06DFA0A4679
:10C03400114607B0F0BD034A0020F9E7FE070000EF
:10C044000000E0FF0000F0FF0000F87F9EA0E63F44
:10C05400CE3B7F660000F0BF0000E0BF0000E03F81
:10C06400C03000089AB5B312FF0750C0A80C615C39
:08C0740010D02BBF0030E63FA5
:10C07C00F0B585B00C4607465948411C220D0A40C4
:10C08C00511E814200D38EE05948C01B5748A04135
:10C09C0000DAA2E000205849C91B5649A1410146CB
:10C0AC007FD30120C007214681435648381A544893
:10C0BC00814174D3544A554B3846214602F017FB44
:10C0CC000122D2072240524BD31800252A46049550
:10C0DC0000F016FA00F05AFC039000F0F9FC029004
:10C0EC000E464C4B002202F002FB3A46234600F06F
:10C0FC0007FA04460F46484A484B0298314602F06C
:10C10C00F6FA22463B4600F0FBF906460D4602467F
:10C11C000B4602F0ECFA0F46414A424B04460290A1
:10C12C0002F0E5FA404A414B00F0EAF922463B4660
:10C13C0002F0DDFA3E4B049C224600F0E1F9324657
:10C14C002B4602F0D4FA05460E46204630492A46C4
:10C15C00334600F0B9FA01900091364A364B029CF6
:10C16C002046394602F0C3FA344A354B00F0C8F980
:10C17C0022463B4602F0BBFA019A009B00F0C0F944
:10C18C0002460B462846314600F002FB049A204B2F
:10C19C0000F0B6F9039A521CFFF756FD01E017495F
:10C1AC00002005B0F0BDF80F610008187900494275
:10C1BC000C49814121460ED30120C00781430A4816
:10C1CC004840384300D075E7002C214600DA0021A6
:10C1DC00002C00DA00273846E3E70349E0E7C046C5
:10C1EC00FE0700000000E0FF0000F07F422E8640BA
:10C1FC00EF39FAFE2B2386C0D2BC7ADD0000F03F6B
:10C20C00A19CC73B2342920C3CF92F9E2C15F73F67
:10C21C000000E03F0030E6BFA80C615C10D02B3F63
:10C22C001CDC586FA452F13EE0F6B36FE4707C3F17
:10C23C000000D03F0938DE6F993F403FB351427147
:04C24C008E71AC3F04
:10C25000F0B585B016460024E7438B4D7A1C2A467C
:10C2600062414A4002436FD001955A00550D00D1FA
:10C2700008E100940290874C601C039104930D0D1B
:10C2800005406D1EA54273D21D461C0D0440824B15
:10C29000E4185B1C9C426BD337463046294600F0BD
:10C2A0007BFB064600F01AFC2A46029D784051406E
:10C2B0000143039C30D101200290C00786422BD05D
:10C2C000002E0096714B41D0F0174640361A0027D9
:10C2D00001970393012E019A00D02A460497012E5C
:10C2E0006A4B00D023462F462846214602F005FA25
:10C2F000224605460C46304602990840634B00D062
:10C30000134642423A400498039902F0F6F9074670
:10C310000B467608DDD11AE0002228462146134656
:10C3200000F01AFB002802D0604900241DE0012023
:10C33000C007844328462146FFF7ECFD3A46049B9C
:10C3400002F0DBF9FFF79AFE04460EE0002700201A
:10C350004E493A461D4600F021FA0446009800284E
:10C3600000D42946002800D43C46204605B0F0BD44
:10C370000298C30F4C00E3184400641E484C5C4113
:10C38000E2D20125F30FD21873005B1B434B9A4195
:10C3900010D23F4A114210D0424B0C465C4004433D
:10C3A00026D00C4654400443049827D100283CDA98
:10C3B0002146DAE734460499D7E737463046049CED
:10C3C000214600F0E9FA064600F088FB4C403B4667
:10C3D0004340234327D1049900291C46194600DA1B
:10C3E0002B49F007C1D0E807039E06407118BCE74F
:10C3F0000094049800281ADA009819E0584006437F
:10C4000002982CD1284A4A400243009C1F49ACD0D4
:10C41000EA07039B93430022391A01989841144676
:10C420002ED31B4A2CE0049A3FE711469DE71046A5
:10C4300003903046049F394600F0AEFA044600F0FF
:10C440004DFB794070400843039802D1E8070399F7
:10C450000818E10700D00390009C039985E7EB07DB
:10C460000C469C430023391A0198A0411C461946EA
:10C4700000D37AE70C48039E46400298304301D02F
:10C48000114672E7014970E7FFFFEF3F0000F03F00
:10C490000000F07FFE07000001F8FFFF0000E0FF52
:10C4A000FFFF1F000000F0FF0000F0BF0000F87F5A
:10C4B000F0B581B000280090124D13D00146C0178E
:10C4C00041400F1A0026104CF80707D00CCC30461C
:10C4D0002946083C02F011F906460D4608347F084B
:10C4E000F2D100E000260020064932462B4600F03B
:10C4F00055F9009A002A00D43046002A00D4294673
:0CC5000001B0F0BD0000F03FE830000882
:10C50C00F0B40125ED070F005F405AD48B4200D1E7
:10C51C00824205D950404240504059404B4059400E
:10C52C004E18760DDF187F0D3BD0741C640529D096
:10C53C00F41B352C26D80E0DDB022B43DB0AC9026B
:10C54C002943C9121700202C1ED2E741E240574064
:10C55C00E3415A40A340E3405A400024801859411B
:10C56C000AD3B21C520521D0C207012F6241170019
:10C57C004008CB0718434908013636054208AF413D
:10C58C0060417141F0BC7047203C06D01F00E74170
:10C59C00E3405F400024012A6741C0186141EBD39E
:10C5AC00DFE7002EEED129400020EBE70136310504
:10C5BC000020E7E7E742E5D10020C143090DC9049B
:10C5CC00E0E76B400E00871A9E4104D26E40C01B00
:10C5DC00B141D21973414E18DF18AC0AE642E9D2C8
:10C5EC00760D7F0D31D0F41B362CCBD8B4460E0D06
:10C5FC00DB022B43DB0AC9022943C90A012C32D8BE
:10C60C0004D1D4075208DF073A435B08EF0A6442AF
:10C61C00904199411ED0002239424DD124194041FC
:10C62C0049410124394204D10134001849413942AD
:10C63C00FAD06246A24204D9361B013E360589194E
:10C64C00A0E7F10AC90700209CE736429AD10020E6
:10C65C00002197E70200224394D0B842DED20100B9
:10C66C0020002024E3D1202C13DD203CE2411700D4
:10C67C00A240E2405740E3415A40A340E3405A40B5
:10C68C00012FBF410137174300227C429841914151
:10C69C000CE01700E741E2405740E3415A40A34009
:10C6AC00E3405A407C429041994100220F0303D24F
:10C6BC00013E241940414941013E36054708AC4131
:08C6CC0050417141F0BC7047C0
:10C6D400F0B40125ED076B40004C204713C500085A
:10C6E40030B405004D400124E407254042004B00CE
:10C6F400120E32D01B0E3CD0FF2A33D0FF2B3FD07A
:10C70400D21800022043000A09022143090AC4B2D4
:10C714004C43000AC3B24B43000A4843210A5B1846
:10C72400190A091801D44900013A080A7F3A2ADB98
:10C73400FE2A0FD2D2051C43240601D00124214332
:10C74400C9B280295041802901D1400840002843C2
:10C7540030BC7047FF20C005F9E71B0EFF2B0AD041
:10C764002800F5E7400206D1FF2BF3D1490202D19C
:10C77400F0E7FF2AF4D17F2000010C300005E7E741
:10C784004902F8D1E6E743020132E9D15B120233F0
:08C79400E6D9D805E4E7C04630
:10C79C00F0B40125ED070C005C402C40A446AE0A19
:10C7AC004C18DF18F4423DD2F74245D2640D4CD000
:10C7BC007F0D3CD0E41BC9022943CF0ADB022B437B
:10C7CC00DB0A0600B61A9F4104D2013CB6197F4120
:10C7DC00B6185F416812800D241838DD00188442A9
:10C7EC0025D8E80C0021B6197F41B61A9F4103D316
:10C7FC0040414941F7D304E0B6185F410018494164
:10C80C00F1D32405B6197F41B61A9F4105D337439E
:10C81C00C20717430022012F504161416246114368
:10C82C00F0BC70470CD100280AD1F74208D2002086
:10C83C00C143490D0905F1E7002A01D1F74206D0A1
:10C84C000020C143090DC904EAE77F0DF8D0002090
:04C85C006146E5E765
:10C8600030B401256D054C00E54215D85C00E54269
:10C8700012D80C001C436400044314430FD005D2AB
:10C8800082428B418041013030BC704790429941D7
:10C890008041013030BC7047002030BC704701201F
:04C8A00030BC7047F1
:10C8A40070B4012676054C005D00E6420CD8EE42D9
:10C8B4000AD825430543154303D0994204D1904235
:10C8C40002D1012070BC7047002070BC7047C04684
:10C8D40030B401256D054C00E54215D85C00E542F5
:10C8E40012D80C001C436400044314430FD005D237
:10C8F400904299418041013030BC704782428B4163
:10C904008041013030BC7047002030BC70470120AA
:04C9140030BC70477C
:10C9180030B401256D054C00E54215D85C00E542B0
:10C9280012D80C001C436400044314430CD005D2F5
:10C9380082428B418041404230BC704790429941CD
:10C948008041404230BC7047002030BC7047C04630
:10C9580030B401256D054C00E54215D85C00E54270
:10C9680012D80C001C436400044314430CD005D2B5
:10C97800904299418041404230BC704782428B418D
:10C988008041404230BC7047002030BC7047C046F0
:10C99800F4464A1805D200F063F801D5C0174008DC
:10C9A800604701235B05D34206D200F059F801D550
:10C9B8000120C0074042604701D10042F5D0D0179E
:04C9C800400870476C
:10C9CC004A00520D01239B02D21A01321DD452424D
:10C9DC003F321DDD8C46C902430D1943C0020123B1
:10C9EC00DB071943202A02D308000021203AD14149
:10C9FC00D04048409140D140484063461B4203D54B
:10CA0C00002340428B4119007047002000217047E1
:10CA1C00002801D0012211434B0001225205D342C0
:10CA2C0000D959080020C90FC90701D4C0434108D7
:04CA3C007047C04639
:10CA400041000DD2090E7F390AD449421F3105D465
:10CA500000020122D2071043C8407047C817704730
:04CA600000207047FB
:10CA64004A0010D2520D03231B02FF33D21A0AD4F8
:10CA740052421F3209D4400DC90208430123DB0787
:10CA84001843D040704700207047D0177047C04605
:10CA94004B001BD25A0D01239B02D21A013215D42A
:10CAA40052423F3215DBC902430D1943C002012330
:10CAB400DB071943202A02D308000021203AD14180
:10CAC400D04048409140D140484070470020002168
:08CAD4007047D0170100704704
:10CADC00054B004206D5404200B5984708BC0122E0
:0CCAEC00D20711431847000075CB00086A
:10CAF8000B00034329D0CA0FD200043212023D3280
:10CB0800094203D5002349424042994102D101001C
:10CB18000020203A0B0C04D1103A0904030C1943E5
:10CB28000004094203D4013A00184941FBD5844660
:10CB3800C00A4B051843C90A120563465B055B41E9
:0CCB480002D3012B0023584151417047DB
:10CB54009D2201000AD002D4013A4900FCD5D20535
:10CB6400080A0906494100D3012950417047C046CB
:10CB740042221201033A010007D002D4013A0018FC
:0CCB8400FCD51205C30A40059918704743
:10CB90000B00034305D0042212023D320942014B2F
:08CBA0001847704715CB00088F
:10CBA800202A07D203009040914052422032D340BD
:10CBB80019437047203A0100914000207047C04651
:10CBC800202A07D2D0400B00D14052422032934055
:10CBD80018437047203A0800D04000217047C046EB
:10CBE800202A07D2D0400B001141524220329340F4
:10CBF80018437047203A08001041C9177047C046CB
:10CC080030B5514343435C18010C130C0D005D43D0
:10CC1800641992B2514380B242430D0C0904521870
:10CC280065415843010C00048018694130BDC04675
:10CC3800CA1751408B1A17D0C1174A40944648402A
:10CC4800411A48081A0000E052008242FCD900202C
:10CC580000E05208914200D3891A40419A42F8D123
:10CC680062465040801A704710B500F095F810BD24
:10CC780007B5FFF7DDFF0EBC4243891A00BDC04669
:10CC88000A0015D00300400800E052008242FCD997
:10CC9800002000E052089B1A06D340418A42F9D18D
:10CCA800704752089B18F8D200188A42F9D1704789
:08CCB80010B500F071F810BD89
:10CCC00038B504004D42FFF7DFFF4543611938BD19
:10CCD00070B5CC1760406140001BA141DD176A4070
:10CCE0006B40521BAB4100F00BF862406340121BDB
:10CCF000A3416C4060406140001BA14170BDC04633
:10CD0000002B09D1002907D110B51100FFF7D8FF7A
:10CD10000A000021002310BD70B400240125ED0796
:10CD2000002B07D1002905D0834203D21300002233
:10CD30002C0000250026A419994200D1904212D956
:10CD400092185B4103D2EE076D086408F3E7DE0733
:10CD50005B08520892190126F6079B1903E0DE07CB
:10CD60005B0852089219801A994103D364416D41BE
:10CD7000F5D30FE024196D410AD2DE075B08520893
:10CD8000921980185941F5D364416D41E7D301E010
:10CD90008018594102000B002000290070BC704728
:08CDA000002000217047C0468D
:10CDA800F0B503AF93B06E46F51D2135F41D393447
:10CDB80074613362F261F160306101F03BFFB06091
:10CDC800C21D07218A436946B1616946881A7060A5
:10CDD8008546F41D1D3400212422204600F0CAFF98
:10CDE8000B487169F2680A6048600A48286030692F
:10CDF8002862B06868617068E8602046F169326A44
:10CE080000F01EF8B1698D46FE1F053EB546F0BD1F
:08CE18002DEC0008FFFFFF7F75
:10CE200083B010B581B0044603A80EC00548006861
:10CE300003AA0092214601F066FD01B010BC02BCBD
:08CE400003B0084718000020B0
:10CE4800F0B59FB012920B460446002020600121E5
:10CE58000A020F924A020B928A020192CA020092B7
:10CE680003220D92920205920D034A0307928A0348
:10CE780003920491C90317910A90C0430290169433
:10CE880009951978252909D0002901D100F03CFE1F
:10CE98005C1C169801F0D6FC2346F2E7DB1C0A9FBF
:10CEA8000B9C981E00780246203A102A2CD8802124
:10CEB80092003E461F4602A39A583B46374697467D
:10CEC8000DCF00082DCF00082DCF000827CF000870
:10CED8002DCF00082DCF00082DCF000821CF000846
:10CEE8002DCF00082DCF000851CF000825CF00080E
:10CEF8002DCF000819CF00082DCF00082DCF00082E
:10CF08001DCF000840210AE05E28294607D009E025
:10CF1800102104E0214602E0179900E020210F4388
:10CF28005B1CBEE75B1E014630390024092916D870
:10CF38000A2161434418303C591C18780246303A9B
:10CF48000A2A0B46F4D30AE0129901C91291C10FBB
:10CF580009010F43C1174840441A581E007800269B
:10CF68002E281CD118782A2805D158789B1C12998C
:10CF780040C912910FE05B1C0146303909290CD8D1
:10CF88000A2171434618303E591C18780246303A37
:10CF98000A2A0B46F4D3002E01D40F990F43E11748
:10CFA8006B2808DC4C2803D068283CD06A280AD1B2
:10CFB8000220074305E06C2830D07A2801D0742875
:10CFC80001D118785B1C8C43462811931BDD014660
:10CFD8006339152937D8C0467944097949008F44FF
:10CFE800710B4D1BD70A0B0A0A0A0A8194610A0AB7
:10CFF8008F0A560A0A3A44E70C94039C27430021F7
:10D00800089139468EE0442815DD452834D0462855
:10D0180000D036E7079807430098BAE018786C28DC
:10D028002ED1022003E0187868282CD10820074365
:10D0380058789B1CC7E7252800D08EE22521169832
:10D0480001F000FC7AE2472800D19FE0582800D080
:10D0580017E707990F430C94D34A782800D1203258
:10D06800039C0F990F42394601D0D04B19403B061B
:10D07800DB171340089355E007980743019888E0A9
:10D088005B1C049A01E05B1C042217439BE70C9489
:10D098000F990F4201D0C5490F403946039C002221
:10D0A80008923FE00C9438060F990F430E97C0176B
:10D0B800232101400891129820C8129000240820CA
:10D0C8000690D3E1129E3578621E169C204639469A
:10D0D800159201F009FC2046294601F0B3FB361DE4
:10D0E8001296C2E01298006839071699096800D5A7
:10D0F80037E2BA07016000D434E20021416031E22E
:10D108001596129901C912918EE00C940F990F424D
:10D11800394601D0A54A11403A06D21730231340A8
:10D128000893039C02220A40214205D1002A129A40
:10D1380008D1131D00240BE0002A129B13D104CB45
:10D14800D41715E0D21D07239A43546813460833B1
:10D15800129315684A0713D408220A4000D0EDB28A
:10D16800002A0ED102E1DB1D0722934314CB0033C2
:10D1780012934B0707D40B0700D5E3E01546E4E00C
:10D18800ADB20024F2E015B21204DDE007980743BF
:10D19800059807430F98074201D0304600E0062063
:10D1A8000C943946059A1140891A4A424A41002886
:10D1B80000D002461592129CE41D0720844326687D
:10D1C800656830462946FEF721FD08341294002888
:10D1D800304629460ED000221346FFF7B9FB3A46DF
:10D1E80007990A4000280C9C0FD0002A704819D0D3
:10D1F800704817E0FEF7FCFC00280C9C37D0079815
:10D2080007426D480ED06D480CE0002A6C4900D0EA
:10D218006C49002A01D06B4800E06948401CBA06F6
:10D2280000D5084668490F400028684E00D00646D9
:10D238000F980742304602D100F016FD02E015991A
:10D2480000F04AFD054659480740621B16983946C2
:10D25800159201F049FB002D07D0169C3178204625
:10D2680001F0F0FA761C6D1EF8D1F8065DE1304643
:10D278002946FEF7D7FC002800D10646002800D131
:10D28800002513963046294601F068FC0446012023
:10D29800002C089001D0C00745401EAA30461095C2
:10D2A8002946FEF7F7FC1E980D9948430A21FFF717
:10D2B800BFFC06461E90002C01D0602007430022C8
:10D2C800139C2046294614921346FFF7E7FA0028D4
:10D2D80018D1701CFFF7E8F822462B46FFF738FBF9
:10D2E80000281E9806D0411C1E91801CF2E71E984B
:10D2F800401E1E90FFF7D8F822462B46FFF708FB82
:10D308000028F4D13D4605980540089883021E98E8
:10D318009D42159E00D113E105998D4207D18642A1
:10D3280000DC0DE10421C943884200DC08E10199D1
:10D338000F42109D0E9300D180E20E2800DCD0E150
:10D34800149E7BE255B21206D417002C05D48A0627
:10D358000AD44A060AD5202207E000226D42A241DB
:10D368002D230893144601E02B2208920F9A1142AC
:10D3780001D00E4A11400A460F990E920A420499AA
:10D3880000D03146069100276E2838DD6F3809280D
:10D3980000D98AE078440079400087441967868676
:10D3A800868636868667C04658300000FFFDFFFF38
:10D3B80044F200083FF20008A8F40008A4F40008AA
:10D3C8004EF2000849F20008FFFEFFFFF7ED0008E3
:10D3D8002846204369D0E80861074018014607201D
:10D3E8002840303018AAD055C808E40862078018C9
:10D3F8000A4622437F1C002A0D46EFD155E05828E3
:10D4080034D0642801D069284FD1284620434CD015
:10D4180011461798014010912A461098002808D004
:10D4280038460D990840032803D118A82C21C15566
:10D438007F1C002510462146159414460A222B46C7
:10D44800FFF75AFC149013910A222B46FFF7D8FBDA
:10D45800201A3021014318A8C1557F1C0920001B40
:10D4680015988541149D139CD6D31EE02846204369
:10D478001AD007980E990142C04800D0C04829091F
:10D488002207891800270A460F212940415C18AB5A
:10D49800D955110924092307C918134623437F1CAA
:10D4A800002B1546EFD100E00027089DFF2D01D87D
:10D4B800029801E0B348FF300B9C0C9B0699CE1BE9
:10D4C800F1178E43B9195A1A002D00D012180E9967
:10D4D800214203D1169801F007FA00221592290A71
:10D4E800169C03D0204601F0ADF901E0002D03D0D1
:10D4F8002046294601F0A6F920460E99159A01F012
:10D50800F3F930212046324601F07EFB012F0ADB79
:10D518007D1C18A84019801E0178204601F092F958
:10D528006D1E012DF5D80E98C006099D119B00D4DB
:10D53800A7E420211698159A01F066FB119BA0E438
:10D548000F9934318842109C06950FD113982146C3
:10D558008D4A8E4BFFF71EF90FE0002800D090E4AB
:10D56800E2E201701298001D12908AE44042FEF730
:10D578009BFF139A234601F0BCF804460E4600228E
:10D588001346FFF78BF9002839D120463146FEF7BC
:10D598003DFB00282046314600D01CE60E970022AD
:10D5A8007B4BFFF793F900281E9F0FD000222046DF
:10D5B8003146774BFFF7EEF804460E460022744BCF
:10D5C800FFF784F97F1C0028F0D11E97002220461F
:10D5D8003146704BFFF7BCF9002811D000222046D5
:10D5E80031466B4B01F085F804460E460022694B24
:10D5F800FFF7AEF97F1E0028F0D11E9700E00E97C6
:10D60800059806998142159801D0014600E0411E0F
:10D61800029D0028149100D1002113914842FEF781
:10D6280043FF2A46FEF712FB22463346FEF76AFFFF
:10D6380006460D4600220692554C2346FFF746F94A
:10D6480000280AD01E98401C1E9000223046294609
:10D658002346FFF79FF806460D4610961595139832
:10D66800002866D000990B4680330E9A13408B42EF
:10D6780061D1102800DB10200546FEF715FF324661
:10D68800159B01F036F8FFF701FA0C4601462143D5
:10D69800069914914FD0214606463F4A3F4BFFF763
:10D6A800AFFA4A08C3079A184008C90708183C493E
:10D6B800081A3C48904114953DD330460A2200236D
:10D6C8002146FFF719FB0C4607460A220023FFF7FD
:10D6D80013FB1498401E14902DD01A433846EDD0F1
:10D6E80029E0C143711810290E4600DB10263A06BE
:10D6F80000D5A3E0002900D1A0E03046FEF7D4FE13
:10D70800139A2B4600F0F5FF00242246264BFEF71D
:10D71800F9FEFEF799FB22461D4BFEF7D7FA224683
:10D728002346FFF7BBF8002800D184E0761EE4D139
:10D7380082E00698149080210E9806460140149ABB
:10D7480011430C98801A002901D1401F00E0801F66
:10D75800139009981E9C064201D1089D46E00321BA
:10D768002046FFF785FA881C0125C04678440079D1
:10D77800400087441B2A381B2A00C04694F400083E
:10D7880084F40008FFFEFFFFA0C8EB85F3CCE17F1F
:10D79800000024400000F03FCDCCCCCCCCCCCCCC8D
:10D7A80099999999999999190000E03F641E1E94D6
:10D7B800002210981599DF4B00F09BFF10901591EF
:10D7C8001398401E139002250DE0A41E1E940022FB
:10D7D80010981599D84B00F08CFF1090159113985C
:10D7E800801E13900325149AD01782437006800F69
:10D7F800149202D01398401E1390204601F000FAAC
:10D80800632802DD1398401E13900898C00237461B
:10D81800874310981599FFF739F906460C46FFF724
:10D82800B3F902460B4610981599FEF74FFF109072
:10D838001591139A76E034461E98264610381496A9
:10D848007142884200DC0846FEF72EFE029AFEF777
:10D85800FDF9139A2B46FEF755FE05460C461E9811
:10D86800401CFEF721FE2A462346FEF7F5FF002856
:10D878001E9800D0401C002814D4112818D3014643
:10D8880010391E911021081AFEF70EFE2A4623466B
:10D8980000F02FFFFFF7FAF806460C460020159017
:10D8A800109018E01095159400261E96344612E044
:10D8B80000201E9028462146FFF7E8F806461594F2
:10D8C8000C46FFF761F902460B4628461599FEF704
:10D8D800FDFE1090159138460E99884397490831F6
:10D8E80000250A4608326D1C0B684968F31A23465E
:10D8F8008B411146F6D280213940149A11434B1EB0
:10D908000A469A41002901D00021C9437B069B0F92
:10D9180000D0D1431E9A891A0C9A149BD21A511816
:10D928004A1B0746D017114681430B9810300E97B3
:10D9380007420AD1012A08DB0F462021169800F079
:10D9480081FF7F1EF9D10E9A01E03A460F4640202A
:10D958001040910603D4002809D0202104E00028B3
:10D9680001D02D2100E02B21169800F06BFF0E98B6
:10D97800C00607D4002F05D03021169800F062FFAA
:10D988007F1EF9D16D1EE8006C4A111849681258BB
:10D99800B01A2046884101D2302007E03020B61A5C
:10D9A8008C41401CB31A23468B41F8D2C1B2169859
:10D9B80000F048FF002DE5D113970E9E34460098DD
:10D9C8000440169F0BD01E98012808DB401E1E90AD
:10D9D8003021384600F036FF1E980028F6DC8020FB
:10D9E80030401499084344D02E21384600F02AFFCD
:10D9F800149D102D00DB1025E8178543002C01D15C
:10DA0800284601E01E98281A159CFEF74DFD149A29
:10DA1800012A22DB109A234600F06BFEFFF736F846
:10DA280004460E462F467F1EF800444A11184968DE
:10DA38001258A01A3046884101D2302007E0302021
:10DA4800A41A8E41401CA31A33468B41F8D2C1B2A6
:10DA5800169800F0F7FE002FE5D11499481B169F81
:10DA68000E9E06D06C1A3021384600F0EBFE641C7E
:10DA7800F9D301980642099D139F38D007980642AA
:10DA880001D0452100E06521169E304600F0DAFEFF
:10DA98001E980028304604D42B2100F0D3FE1E988F
:10DAA80005E02D2100F0CEFE1E9840421E9064280D
:10DAB8000DDB6421FFF7E4F801463031304600F011
:10DAC800C1FE1E986421FFF7D3F808461E910A216B
:10DAD800FFF7AEF801463031304600F0B3FE1E982D
:10DAE8000A21FFF7C5F83031304600F0ABFE002FB1
:10DAF800119B01D1FFF7C5F9169C2021204600F0A3
:10DB0800A1FE7F1EF9D119E5169CE068002805D012
:10DB180006CC083C914201D20A9A4254204600F0B1
:10DB2800D6FE20681FB0F0BD169800F0D0FE02980F
:10DB3800F8E7C04600002440000059403031000892
:10DB480009490968091A4A1E9141084A1268121AB5
:10DB5800531E9A410A4006490968081A411E88411D
:10DB6800104040427047C046180000201C000020AA
:04DB78002000002069
:10DB7C000F480321016141610E4A82610E49C16166
:10DB8C00012189020162002181624162C162026647
:10DB9C000A4A4266102282660167C1664167084ADA
:10DBAC000F234B40D35C4354491C1029F8D17047C8
:10DBBC00FC09002064F20008CA0F00204A1400205F
:04DBCC0053F2000808
:10DBD000F0B581B00D461821414316484618F06A49
:10DBE000183602281ED0144601280ED0002700281F
:10DBF0001DD1304600F099FEA04218D33046294688
:10DC0000224600F09DFE274611E0304600F08DFED2
:10DC10000746A04200D32746304629463A4600F040
:10DC20008FFE04E03046294600F0A7FE074638463E
:08DC300001B0F0BDFC09002069
:10DC3800F0B581B014460D4606460A48007800281B
:10DC480001D1FFF797FFEFF31087012181F31088C7
:10DC5800304629462246FFF7B7FF87F3108801B000
:08DC6800F0BDC046FC090020DC
:10DC7000F0B581B00178002925D003220146009239
:10DC800091430D680023DC438607F60EB440E4435D
:10DC90002C43114D6719A743104A174206D14C680F
:10DCA00067191646A643091D3E42F8D022060FD03A
:10DCB0002204120E09D02202120E08D0220E009B5E
:10DCC00006D0042304E0002004E0012300E0022346
:10DCD000C918081A01B0F0BDFFFEFEFE80808080EA
:10DCE000F0B581B00022002934D00378002B31D068
:10DCF00003270246BA430024E5438607F60EB540E3
:10DD0000EE431568354306463E40711804290CD38E
:10DD10000097134EAF19114BAB433B4204D1091F7F
:10DD20005568121D0329F5D8009F2B060DD02B0432
:10DD30001B0E07D02B021B0E06D02B0E00D0042783
:10DD40003C4602E0012400E002248C4200D30C4651
:10DD5000101A0219104601B0F0BDC04680808080C4
:04DD6000FFFEFEFEC6
:10DD6400002A03D0013A8B5C8354FBD17047C04630
:10DD740000220B0011001A00002A02D0013A81543B
:04DD8400FCD1704717
:10DD8800002A09D0884207D007D280188918524241
:10DD98008B5C83540132FBD17047013A8B5C83540E
:04DDA800FBD17047F4
:10DDAC0002480068002800D101487047580F002035
:04DDBC000000002043
:10DDC0007F2805D8034A125C0348405C1040704726
:0CDDD00000207047ACF40008CEF2000800
:10DDDC007F2805D8034A125C0348405C104070470A
:0CDDEC0000207047ACF40008CEF20008E4
:10DDF80002000000040000000800000010000000FD
:10DE0800FDFFFFFFFBFFFFFFF7FFFFFFEFFFFFFF38
:10DE180000000000040000000200000008000000EC
:10DE280001000000020000000400000006000000DD
:10DE3800080000000A0000000C00000010000000AC
:0CDE4800200000004000000080000000EE
:10DE540000000000000000000000000000000000BE
:10DE640000000000000000000000000000000000AE
:10DE74000100000002000000030000000400000094
:10DE84000600000007000000080000000900000070
:10DE9400000000000000000000000000000000007E
:10DEA4000100000002000000030000000400000064
:0CDEB400D5F00008E0DE0008C0DE000829
:10DEC000C1DD000851EC000807EA0008DDDD0008AC
:10DED0005DEC000815EA000841EC0008D9E90008EB
:10DEE000D7F00008CDF20008CDF20008CDF200080E
:10DEF000CDF20008CDF20008CDF20008CDF2000806
:10DF0000CDF20008CDF20008FFFFFFFFFFFFFFFF8B
:10DF1000FFFFFFFFFFFF00009BF000087FF20008FB
:10DF2000FEED00089CF2000855EE00086DF20008B6
:08DF300076F200085CEE000827
:10DF3800034C206804348047FBE7FCF7C5FCFEE788
:04DF48002CF50008AC
:10DF4C0004480549884385460448804704480549E8
:10DF5C000160EBE70080002007000000C1E600082C
:08DF6C0008ED00E000300008A0
:10DF7400FEE7FEE7FEE7FEE7FEE7FEE7FEE7FEE775
:10DF8400FEE7FEE7FEE7FEE7FEE7FEE7FEE7FEE765
:10DF9400FEE7FEE7FEE7FEE7FEE7FEE7FEE7FEE755
:10DFA400FEE7FEE7FEE7FEE7FEE7FEE7FEE7FEE745
:0CDFB400FEE7FEE7FEE7FEE7FEE7FEE703
:10DFC000F0B581B000904C000120640C0446054679
:10DFD000064610D10C04240E01D000240BE00C06E0
:10DFE00005D44C0606D000242546264603E000242E
:10DFF000254600E0044603231746DF41032F10D8CF
:10E000007F443F797F00BF4403010E11002C08D1EB
:10E010000098006841618168182399431143816029
:10E02000002001B0F0BD002DF2D0FAE7002EEFD0B5
:02E03000F7E710
:0AE0320080B5806A00F00FF880BD91
:10E03C0080B5806A816D40220A438265C16D0422DD
:0AE04C000A43C26500F001F880BD30
:02E05600704711
:02E0580070470F
:02E05A0070470D
:10E05C00F0B587B01346022545770468A2680127FE
:10E06C003A43A260026A012A0FD0022A20D0032A66
:10E07C002CD1002B00D147E11D461540042B0697EF
:10E08C000591039043D2002250E005919E0821D0C7
:10E09C0003223146019211400291711E0329069709
:10E0AC000390049300954FD20027059A019880E0C5
:10E0BC0005915E08069720D00493032135460D4048
:10E0CC00731E032B00D3C8E00027E7E0477700203E
:10E0DC0007B0F0BD0021059E1A4603231A40032AFF
:10E0EC0000D0B2E00B463B43F35C2A46755C2D0234
:10E0FC00EB1823800A43B15CACE00021059EDA07E3
:10E10C0000D1EAE04900715A2180069FFCE093435C
:10E11C0000220E463768276077682760B76827604B
:10E12C00F76827601036121D9342F3D1002D00D1F1
:10E13C00DEE0069B9100059842582260012D00D02C
:10E14C00D9E01F460398DFE0104696430027059A56
:10E15C00D15D0D06D1194B781B045B198D782D02FE
:10E16C005B19CD785B1923600B791B064D792D0457
:10E17C00EB188D792D025B19CD795B1923600B7A25
:10E18C001B064D7A2D04EB188D7A2D025B19CD7A76
:10E19C005B1923600B7B1B064D7B2D04EB188D7BD1
:10E1AC002D025B19C97B59182160361F1037002EC0
:10E1BC00CED1029900291646009D3CD0F15D09068E
:10E1CC003B46069A1343F35C1B0459183B462B43FE
:10E1DC00F35C1B02C9183B460343F35CC91821606E
:10E1EC000299012927D0391D735C1B0628460D4660
:10E1FC001543755D2D04EB180D460543755D2D0219
:10E20C005B19054601980143715C5918216002990C
:10E21C00022910D00837F15D09063B461343F35C25
:10E22C001B0459183B462B43F35C1B02C9180743CC
:10E23C00F35DC9182160049A114681430398069F27
:10E24C0003231A40032A00D14CE7022A47D0012AA3
:10E25C0001D1715C2170046856E08E43059A083236
:10E26C000027931F1B881146083909880904C9180F
:10E27C002160911E0988131F1B881B0459182160EB
:10E28C00518813881B0459182160D18893881B046A
:10E29C005918216010323F1DBE42E2D1002D059E5F
:10E2AC0014D0BA00B1184B88B25A1204D21822609A
:10E2BC00012D0BD0CA888B881B049A182260022D62
:10E2CC0004D04A890989090489182160049B1946DC
:10E2DC00069A9143DA0700D014E7069F14E00B4628
:10E2EC003B43F35C715C0902C918218004680BE0A4
:10E2FC000398069F08E009184A682260022D1F4601
:10E30C00039801D08968216021684777084607B0D7
:02E31C00F0BD52
:0AE31E0000690840411E8841704765
:02E3280070473C
:10E32A00F0B583B004462820205C012802D10220DF
:10E33A0003B0F0BD234628330220587001271F700E
:10E34A00002A0097029306D0C87800044A7812027D
:10E35A0017188E783AE04878C20603D5EF221040A3
:10E36A000A304870CA7800260A2A0FD30A3AD3B26A
:10E37A00CD255D43EB0A0A255D43521B1B01103371
:10E38A001343DAB20A2804D233460CE0D2B20A287E
:10E39A00FAD30A38C3B2CD255D43EB0A0A255D4399
:10E3AA00401B1B01103312040343D8B207028878BA
:10E3BA000A2809D30A38C3B2CD255D43EB0A0A25D8
:10E3CA005D43401B1E011036174306432068CA22CC
:10E3DA004262532242620A78C168490601921CD4F9
:10E3EA00C16880220A43C260F4F733FF05462068F9
:10E3FA00C168490611D4F4F72CFF401B7D21C900DE
:10E40A008842F4D90320029B58702168CA68FF2207
:10E41A004A620021197003B0F0BDF1B20F430199AD
:10E42A004903C02297430F4347602046F6F751FF3E
:10E43A002168FF224A620028029BEAD1009858709C
:0AE44A0000200021197003B0F0BD9E
:02E4540070470F
:02E4560070470D
:02E4580070470B
:02E45A00704709
:02E45C00704707
:02E45E00704705
:02E46000704703
:02E46200704701
:02E464007047FF
:10E4660030B5816ACA070CD18A0714D44A071CD46E
:10E476000A0724D4CA062CD48A0634D44A063CD4C5
:10E486004CE00122520403685C689443C26A22434A
:10E496005A608A07EAD50122120403685C6894432D
:10E4A600026B22435A604A07E2D5012292040368AE
:10E4B6005C689443426B22435A600A07DAD501220C
:10E4C600D20303685C689443826B22435A60CA068F
:10E4D600D2D50122120303689C689443C26B22437F
:10E4E6009A608A06CAD50122520303689C6894433F
:10E4F600026C22439A604A0610D50122130502686F
:10E5060054689C43456C2C4354609D4206D10323BA
:10E516005B0554689C43836C23435360090607D507
:10E526000121C904026853688B43C06C18435060CC
:02E5360030BDF6
:10E5380030B580214158212918D102465632938A94
:10E54800002B13D0016802E05B1E1C040ED0148857
:10E55800002C0CD0CC692406F6D5046D25788D6284
:10E56800641C04651488641E1480EDE730BD012026
:10E57800C0058A6882438A600868402202430A60AC
:02E5880030BDA4
:10E58A0010B580214258212A0DD1024656321388ED
:10E59A00002B09D00168036D1C788C62591C016537
:10E5AA001088401E108010BD006802688A4302600D
:0AE5BA00016840220A43026010BD10
:10E5C40010B584214158222901680FD102465E32D8
:10E5D40053884C6A1C40836D1C801488641E14800C
:10E5E4009B1C83651288002A05D010BD8869082207
:10E5F40002438A6110BD0246843209235B010C6820
:10E604009C430C608B680124A3438B600021C1668A
:0AE614002021116000F031F810BD64
:10E61E0010B5842141582229016810D102465E327C
:10E62E005388496A1940836D19701188491E1180EB
:10E63E00816D491C81651188002905D010BD88693E
:10E64E00082202438A6110BD01468431092252011B
:10E65E0003681C6894431C609A680124A2439A6064
:0EE66E000022C26620220A6000F002F810BDF1
:02E67C007047E5
:02E67E007047E3
:10E6800030B57C21415C012901D1022030BD024618
:10E690007C322421516001680B680C680125AC4371
:10E6A0000C606C07A3430B600021416611702020B1
:06E6B0005060002030BDA7
:02E6B6007047AB
:02E6B8007047A9
:02E6BA00FEE779
:02E6BC007047A5
:02E6BE007047A3
:02E6C0007047A1
:10E6C20008D1002806D1F54204D801D3002A01D18D
:10E6D2006D0D09D10020C143090DC904F0BDF9D166
:10E6E2001242F7D1640DF5D00020C1434905490813
:10E6F200A6E000206146F0BDF0B50127FF070E003D
:10E702005E403E40B446BE0A4C18DD18F442D7D2F1
:10E71200F542E4D2640DECD06D0DEAD06419C90261
:10E722003943460DC0023143DB023B43DB0A10B4DE
:10E732008E4685B297B26F43140C6C433E0CA419FB
:10E74200260C2404BFB227439CB26C43A419190CB3
:10E752006943250CA4B249190D04090C6419000C73
:10E7620095B245433E0C76193743BFB2360C150CB1
:10E772004543AD19A6B2240CAD192E0437432E0C15
:10E7820036199DB24543AD19ACB22E0C89191D0C38
:10E7920045436D182E04290C3443704680B295B25D
:10E7A20045433E0C76193743BFB2360C150C454330
:10E7B200AD19A6B2AD19240C2E0437432E0C36190E
:10E7C2009DB24543AD19ACB22E0C89191D0C4543BF
:10E7D2006D182E043443290C75462D0C90B26843F3
:10E7E2003E0C80190604BFB23E43070CA0B23F188C
:10E7F200120C6A43D019020C80B2240CA4189AB2EB
:10E802006A43121914042043120C89181B0C6B431F
:10E81200C91810BC01273D05294203D1B619404150
:10E822004941013CFF077D0D013D641B0BDB6D007F
:10E83200AC4209DA240500254208BE416841614123
:0AE8420066463143F0BD54E74EE78F
:10E84C0030B581B0044668460170206900280FD0AD
:10E85C000CCC083C9A4233D26269531C63618154DC
:10E86C00A069616981422BD1204600F02EF827E087
:10E87C00E068002809D00CCC083C9A4220D2551CE8
:10E88C009D4200D1002181541AE0A068002808D0D4
:10E89C000CCC083C9A4213D2551C9D420DD0C9B2E7
:10E8AC000CE0236A002B0BD003CC083C884207D227
:10E8BC00694601222046984702E0002192008150CF
:0AE8CC002068401C206001B030BD40
:10E8D60010B54269002A07D00446036A002B01D00E
:0AE8E600216998470020606110BD11
:10E8F00080B5CB0606D4890501D5302100E0202162
:06E9000000F086F980BD65
:10E9060070B514460D460646FFF74DFA01463046E9
:0AE916002A462346FEF745FA70BDBD
:0AE9200080B50068FFF788F980BD9C
:10E92A00C2680169914201D9D04302E0D2438918F1
:06E93A0080680818704718
:10E94000F0B581B0154604464068A268E6688019B3
:10E95000971BBD4204D22A46FFF704FA751909E055
:10E960000E463A46FFF7FEF9F119ED1B60682A469C
:0AE97000FFF7F8F9E56001B0F0BD13
:10E97A00F0B583B016460D46C76800210190029192
:10E98A000269F943BA4202D95418816802E052185E
:10E99A00816854184268C91B8C4200D30C46B442A1
:10E9AA0000D33446D01929462246FFF7D6F9E7198B
:10E9BA00019881688F4200D100270299C760361BEF
:0EE9CA002D196118002EDAD1084603B0F0BDF9
:10E9D80010B50446002000290DD0002A0BD0097874
:10E9E80048B2002808D4002C00D02160002119600A
:0EE9F8005960411E884110BD0120C04310BD72
:0EEA0600014641391A2901D2202108437047E8
:0EEA1400014641391A2901D2202108437047DA
:10EA2200010002000400060008000A000C001000A9
:06EA3200200040008000FE
:10EA3800B0B50146806A836D826D5024234206D0AA
:10EA4800D20610D4006D426B08469047B0BD012134
:10EA58004B021A4382650268D3681B059B0F05D0D9
:10EA6800FCF7A0FAB0BDFFF7F2FAB0BD837E002B29
:10EA7800F6D113681B07F3D593685B070AD40346DE
:10EA8800583354680C25AC435460FF2402341A6888
:10EA9800A24306E0826D20231343836503465C335B
:0CEAA800C26D0A431A60FCF77DFAB0BD95
:10EAB400002A02D0182281507047282281507047C2
:10EAC40042690B4693430A401104C9188161704797
:10EAD40070B582B015460A4604460120C143DE1EC5
:10EAE4008E4200D318460090022D01D3092100E084
:10EAF4000A2108180190069920462B46F8F730F9A8
:10EB0400262000212154A184E16121841C34A171B7
:04EB140002B070BD1E
:04EB1800007D7047C5
:08EB1C0080B5FAF763F880BD33
:0CEB240080B501204002F5F7E3FE80BD43
:10EB3000F0B581B01E4615460C4607461846FFF74D
:10EB400003F80146002000290AD46543A54207D3F3
:10EB5000304639462A46FFF7E3FE2146FEF794F891
:04EB600001B0F0BD53
:04EB6400C80F70471F
:10EB6800F0B581B01C4615460091CA0017183E46FC
:10EB7800103EB068F1682A46FFF7BBFD0CCEFDF7E2
:10EB8800C1FC009A032A0DDB183F561E2A4623466D
:10EB9800FFF7AFFD0CCF083FFDF7B4FC761E083F2A
:10EBA800012EF3D82A462346FFF7A3FD01B0F0BD96
:10EBB800F0B581B01D4616460346C800022916DB8B
:10EBC80000931F18083F4C1C304629460CCF083FBD
:10EBD800FDF798FC32462B46FFF78BFD641E083F75
:10EBE800022CF3D8009B083306460D4600E01B189C
:10EBF800083B0CCB30462946FDF784FC01B0F0BD3C
:08EC0800C1174840401A704793
:10EC100070B5012A09DB0C460546561C28462146DC
:0CEC2000FFF714FE761E012EF8D870BD20
:10EC2C0010B50C46436A01212046FFF77BFF10BD4F
:04EC3C0040207047BD
:10EC4000024601207F2901D9C043704711707047E7
:0CEC5000014661391A2900D220387047B3
:0CEC5C00014661391A2900D220387047A7
:10EC68004552524F52205452494D4D494E47205615
:07EC7800414C5545530A0011
:0FEC7F0049205265666572656E7A3D25660A000A
:0BEC8E00547368756E743D25660A0023
:10EC99002D2D2D204761696E2044726966742043C9
:07ECA900414C202D2D2D0030
:0FECB00041637475616C20543D256620430A0052
:10ECBF0041637574616C20493D2566204128776951
:10ECCF0074686F7574206761696E2074656D70204C
:10ECDF00647269667420636F7272656374696F6EB4
:03ECEF00290A00EF
:10ECF2004B6F7272656B74757266616B746F723D85
:10ED02002566205B2031202F2043656C7369757363
:03ED12005D0A0097
:10ED15004552524F52204144535F313236305F499C
:0FED25006E7075744D757853656C6563740A0074
:10ED340046697273742073746172742064657465B7
:07ED440063746564210A00FD
:0FED4B004953454E534F523A20496E69740A009E
:10ED5A00466C617368206F6220756E6C6F636B20FE
:07ED6A006572726F720A006E
:0FED7100466C61736820206C6F636B65640A00E9
:10ED80002E2E2E466C61736820756E6C6F636B65FA
:03ED9000640A0012
:10ED93004F5554505554535F4C56505F5348554E3E
:10EDA300545F4F56455254454D5045524154555268
:03EDB300450A000E
:0FEDB6004F5554505554204C5650204F4B0A0087
:10EDC5004F5554505554535F4F56505F5348554E09
:10EDD500545F4F56455254454D5045524154555236
:03EDE500450A00DC
:0FEDE8004F5554505554204F5650204F4B0A0052
:07EDF700286E756C6C290009
:10EDFE004A616E75617279004665627275617279EB
:10EE0E00004D6172636800417072696C004D6179EA
:10EE1E00004A756E65004A756C79004175677573A9
:10EE2E00740053657074656D626572004F63746F24
:10EE3E00626572004E6F76656D6265720044656341
:07EE4E00656D6265720000B2
:07EE5500414D00504D00008B
:0FEE5C0025612025622025652025542025590099
:0EEE6B0075617274206572726F72200A0D005C
:10EE79002D2D2D204761696E202043414C202D2DD9
:02EE89002D005A
:10EE8B004144535F313236305F426174746572793D
:10EE9B0043757272656E744761696E43616C69622A
:10EEAB00726174696F6E53746172743A2045525279
:10EEBB004F5220494E2043414C4942524154494FF5
:10EECB004E2C204E4F205245464552454E43452031
:0AEEDB0043555252454E54210A00DF
:0AEEE50054736869703D25660A0049
:10EEEF002D2D2D204761696E202043414C20454E2A
:06EEFF0044452D2D2D00FD
:0EEF050064656C746120543D256620430A004B
:0AEF130052656620493D25660A009C
:10EF1D004E6F726D616C20737461727420776974B9
:10EF2D00686F757420454550524F4D206368616E72
:0EEF3D006765732064657465637465640A001B
:10EF4B00454550524F4D2046554C4C20524553543D
:06EF5B004F5245210A009F
:10EF6100454550524F4D2053544F524520434F4E2B
:06EF7100464947210A0099
:0EEF77004144533132363020496E69740A002D
:10EF85002E2E2E456E61626C65206C6F636B20655D
:06EF950072726F720A00A7
:10EF9B002E2E2E466C617368206C6F636B20616C38
:0EEFAB007265616479206163746976650A009D
:10EFB9002E2E2E466C617368206F6220756E6C6F01
:06EFC900636B65640A00A1
:10EFCF00466C617368204F7074696F6E62797465F7
:10EFDF002070726F6772616D6D206661696C656418
:02EFEF000A0016
:10EFF1002E2E2E44697361626C65206C6F636B20E9
:10F0010070726F636573732066696E697368656496
:02F011000A00F3
:10F013004F5554505554535F4C56505F42415454CE
:10F023004552595F554E444552564F4C54414745FE
:02F033000A00D1
:10F035004F5554505554535F4C56505F43484950B3
:10F045005F4F56455254454D5045524154555245D2
:02F055000A00AF
:10F057004F5554505554535F4F56505F434849508E
:10F067005F4F56455254454D5045524154555245B0
:02F077000A008D
:10F079004F5554505554535F4F56505F434849506C
:10F089005F554E444554454D50455241545552459E
:02F099000A006B
:10F09B0053756E646179004D6F6E646179005475C0
:10F0AB006573646179005765646E6573646179009B
:10F0BB005468757273646179004672696461790092
:0AF0CB0053617475726461790000EE
:02F0D5004300F6
:02F0D7002E0009
:10F0D90056616C7565206E6F742076616C69640A7F
:01F0E9000026
:10F0EA004672657175656E6379204D6561737572D7
:09F0FA006564203D2025640A0034
:10F10300492028776974686F757420636F6D706523
:0DF113006E736174696F6E293D25660A00F8
:10F120004552524F52204144535F313236305F5383
:10F130006574496E7465726E616C52656665726560
:05F140006E63650A008A
:0DF1450057726974696E6720534E210A00ED
:10F15200554E4B4E4F574E20434F4D4D414E440A54
:01F1620000AC
:10F16300537461727420656E61626C6520726561AF
:10F17300646F75742070726F74656374696F6E0A5F
:01F18300008B
:10F184002E2E2E466C61736820756E6C6F636B0A4D
:01F19400007A
:10F19500466C617368204F7074696F6E627974652F
:09F1A500206C6F636B65640A00C5
:10F1AE002E2E2E456E61626C65206C6F636B207027
:10F1BE00726F636573732066696E69736865640A3E
:01F1CE000040
:10F1CF00466C617368204F7074696F6E62797465F5
:0DF1DF002070726F6772616D6D65640A00CB
:10F1EC004F5554505554535F4C56505F4F564552E3
:09F1FC0043555252454E540A00DD
:10F205004F5554505554535F4F56505F42415454D7
:10F215004552595F4F564552564F4C544147450A42
:01F2250000E8
:10F226004F5554505554535F4F56505F4F564552A5
:09F2360043555252454E540A00A2
:05F23F002D494E4600C0
:05F244002D696E66005B
:05F249002B494E4600B8
:05F24E002B696E660053
:10F2530000000000000054545220524547474553D4
:01F2630000AA
:09F264005465726D696E616C0065
:09F26D00256D2F25642F25790081
:09F2760025483A254D3A255300C4
:10F27F0053756E004D6F6E005475650057656400D1
:0DF28F0054687500467269005361740000F8
:10F29C004A616E00466562004D61720041707200F9
:10F2AC004D6179004A756E004A756C0041756700B6
:10F2BC00536570004F6374004E6F760044656300B5
:01F2CC000041
:01F2CD000040
:0DF2CE0000070320041702010857104080BC
:01F2DB00FF33
:04F2DC00EDB6000883
:10F2E0004552524F52204144535F313236305F53C2
:0CF2F000657444617461526174650A0029
:10F2FC004B6F7272656B74757266616B746F723D75
:04F30C0025660A0068
:10F310002D2D2D204761696E20447269667420434B
:0CF32000414C20454E4445202D2D2D0071
:10F32C004552524F52204144535F313236305F5375
:0CF33C00657443686F704D6F64650A00D3
:10F34800454550524F4D20776173206368616E6761
:10F35800656421205765206E65656420746F207090
:10F36800726573657276652063616C696272617437
:10F37800696F6E20616E642073657474696E67735B
:08F388002064617461210A0098
:10F39000454550524F4D20464143544F52592052FB
:10F3A0004553544F52452F555044415445210A006E
:10F3B0007265616420636F6E6669672E2E2E0A0087
:10F3C000666163746F727920726573746F72652EF3
:04F3D0002E2E0A00D3
:10F3D400466C61736820756E6C6F636B2065727226
:04F3E4006F720A003A
:10F3E80050524F54454354494F4E3A204F425F5272
:0CF3F80044505F4C4556454C5F300A0005
:10F4040050524F54454354494F4E3A204F425F5255
:0CF4140044505F4C4556454C5F310A00E7
:10F4200050524F54454354494F4E3A204F425F5239
:0CF4300044505F4C4556454C5F320A00CA
:10F43C004F5554505554535F4C56505F5348554E8E
:10F44C00545F554E44455254454D504552415455C8
:04F45C0052450A000B
:10F460004F5554505554535F4F56505F5348554E67
:10F47000545F554E44455254454D504552415455A4
:04F4800052450A00E7
:10F4840030313233343536373839414243444546D6
:10F494003031323334353637383961626364656606
:04F4A4004E414E0087
:04F4A8006E616E0023
:10F4AC0020202020202020202068282828282020E8
:10F4BC002020202020202020202020202020202040
:10F4CC0048101010101010101010101010101010F8
:10F4DC008484848484848484848410101010101098
:10F4EC0010818181818181010101010101010101F1
:10F4FC0001010101010101010101011010101010A5
:10F50C0010828282828282020202020202020202C1
:10F51C000202020202020202020202101010102069
:10F52C0079F5000829000020311400008BF5000843
:10F53C00000000204CF500082900000043DF000803
:10F54C00B4DE0008B4DE0008B4DE0008B4DE000847
:10F55C00B4DE0008040000004C0F0020500F002007
:0CF56C00540F00200024F40001000000F7
:10F57800206861680834002200E042540139FCD553
:02F588007047CA
:10F58A0020686168A2680C3401E08B5C8354013AFC
:04F59A00FBD57047E6
:10F59E00FFFFFFFFFFFFFFFFFFFFFFFFFFFFFFFF6D
:10F5AE00FFFFFFFFFFFFFFFFFFFFFFFFFFFFFFFF5D
:10F5BE00FFFFFFFFFFFFFFFFFFFFFFFFFFFFFFFF4D
:10F5CE00FFFFFFFFFFFFFFFFFFFFFFFFFFFFFFFF3D
:02FFFE00FFFF03
:020000040801F1
:10000000FFFFFFFFFFFFFFFFFFFFFFFFFFFFFFFF00
:10001000FFFFFFFFFFFFFFFFFFFFFFFFFFFFFFFFF0
:10002000FFFFFFFFFFFFFFFFFFFFFFFFFFFFFFFFE0
:10003000FFFFFFFFFFFFFFFFFFFFFFFFFFFFFFFFD0
:04F7FC005A89EAFB41
:040000050800DF4DC3
:00000001FF
